:020000041100E9
:10300000002373B52B4D2C4C28006361022601F080
:1030100073F94021FE2221742800284B009601F00C
:10302000BDF9002836D1217CFF222800244B0096D0
:1030300001F0B4F900282DD1224BA2899A4226D161
:10304000E389214A93420DD1204B6361204B2268D2
:10305000002A03D1002B01D043CB43C4280001F048
:1030600089F973BD1B4A934201D00023EFE71A4B45
:103070001A4A1B68934206D9C02304222800217CE7
:103080009B0001F001FA114B6361154BDFE7002350
:103090002374EAE7CC233821AC2228009B01217459
:1030A00001F0F2F90028F2D10E4B63610E4BE3817F
:1030B0000E4BCCE7F441FF1F9061FF1F9C61FF1F87
:1030C0009E61FF1F59590000830500002541001132
:1030D00048B9001182150000B461FF1F871300007A
:1030E00054B90011DD410011AAAAFFFF3CB900113B
:1030F000F7B5164B0192C318021D002000938823D8
:103100005B05D3181B685C1C1AD09CB2402C18D8E5
:103110008D781E0CAC466746CD782D023D43AE42FD
:1031200006D1019800280ED110000C70240A4C70B2
:1031300003249BB20733A343D218009B9A42DED3E9
:10314000FEBD4432F9E71000FAE7C046FC0F00006C
:10315000802213B503000324019189B25201073183
:103160009B18A14304305A1A88235B05C3181B68B7
:10317000591C03D190429241104016BD99B240298A
:1031800007D80B000733A343C0189042ECD30020AC
:10319000F3E74430F9E7134B134A1B68126810B584
:1031A000FA24934201D81A00F824104BE4021B6859
:1031B0009A4210D813000E4A12689A420ED3013375
:1031C00007D1F823DB029C4203D10A49054808F0E5
:1031D00017FB200010BDFC24E402ECE7FE24E4020F
:1031E000F7E7C04600C0071100D0071100E0071143
:1031F00000F00711FFFFFF7FF0B59BB015000490B2
:103200000391402A00D9A0E006AB59801A80FFF74D
:10321000C2FF0400042816D9002206A9FFF768FFA0
:10322000052810D906AB1B88AB420CD1002D07D066
:10323000514B2A000499C01808F0A2F9002802D1C5
:1032400001201BB0F0BD06AB1D8020000699FFF7E2
:103250007FFF041E7BD1069B0793FFF79CFF802313
:103260005B01C618802307001B039E4201D3F8268A
:10327000F60288235B05F31801931B68013302D023
:10328000019808F0D5F83D49019808F0B9FA3B1DBE
:103290000293331D05938822029B52059B181B68DD
:1032A00008935A1C3CD044219AB20091402A04D879
:1032B0000320D11D814389B2009103991B0C8B42DD
:1032C00024D0402A22D80122300008A9FFF710FF9D
:1032D000021E1BD1380008A9FFF70AFF04000428CA
:1032E00031D9009A059B9B1880225201B218934253
:1032F00040D288235B05C118009A09A808F068FA33
:103300001D4B009A09A9F01808F0C2F8009A029B18
:103310009446634402931A4B029AFB189A42BAD31A
:1033200088235B05FC1821680198013908F068FAC8
:10333000200008F07DF8039A07AB5A803000079907
:10334000FFF706FF0400002C03D1002079E70428D2
:10335000FBD988235B05E018069908F051FA03238E
:10336000EA1C9A4300D16BE7034B0499E01808F07C
:103370008FF865E70424ECE704000011FFFFFF7FEE
:10338000F80F0000F7B505001400402A21D80027E7
:1033900001AE71803780FFF7FEFE042816D93A008F
:1033A0003100FFF7A5FE042810D93688BC420BD0A7
:1033B000BD4209D0221CB44200D9321C064B92B245
:1033C000C118280008F004FA30B2FEBDC04300B2B4
:1033D000FBE703204042F8E70400001137B5042260
:1033E00004000D0001A81649FFF7CCFF02000428D5
:1033F0000BD1019BA34208D3AB4204D0104901A8D2
:103400000195FFF7F9FE01203EBD0E4C2368200018
:10341000019308F00DF8019920000139019108F09D
:10342000EFF980235B01E418074B9C42EED10422A4
:10343000034901A80195FFF7DFFE0020E4E7C0463D
:103440005555000000C007110000081130B589B0C3
:1034500008F01EF910226946254807F019FF254B90
:10346000009A9A420ED1019B029A0F2B33D8002169
:1034700001240698013B08D2002900D00292029B49
:10348000013331D10023029325E0551CF2D1020013
:103490002100EFE710341022200004A907F0F8FE05
:1034A000029B013301D1069B0293882304995B059B
:1034B000C918059B06981A03120B049105928142C4
:1034C00003D02B4201D108F083F9019B013B01930A
:1034D000019B002BDED1029B002B03D004930498A8
:1034E0004168084709B030BDE025014C2D03EFE7E6
:1034F00000000111504859368022F8B5964C974B80
:10350000D200002120001C6007F032FF2300944A03
:1035100088331A60934B1A786A23002A00D011333B
:10352000E3620A232365904B37221B780820A363AC
:103530008E4B2118E361102323628D4B3B25636181
:10354000C823DB00A36123008C331A602823013ACF
:10355000E26320646364CA67043A211DCA672100DC
:10356000BC310D602100C03108602100C4310B6006
:1035700021000635CC310D602100083DC8310D60B9
:103580002100D0310A602200D43210602200D832EB
:10359000136022000227E032210017604222DC3152
:1035A0000A6021001B3DE4310D602100E831086014
:1035B0002100EC310B6023000521F4331960230056
:1035C000F0331A602300183290331A6023009433CA
:1035D000186023001E3A98331A60AF23DB00236083
:1035E000644BFA262363644B644DE360644BF03113
:1035F000A3642300FF31FC33B600A16021611E608B
:10360000A5627325E5656D3D6565A56596255D4AF1
:10361000AD00E264666258606766A566002709250A
:10362000A767E566584F594D606720002567E26738
:103630003A6015279C30676007001A203860200028
:10364000A0300700212038602000A83007004C4837
:1036500038602000F830066026006427A436376002
:1036600026005F3FAC3637602600033FB036376038
:103670002600C637B436376026000027B8363760D4
:1036800038269E60424E96205E64424E5A66DE6147
:10369000414E9A645E62F53EFF3E9E621E269A6728
:1036A000354A8000DE661F675F67DD651D6618624C
:1036B000DA67BE23394A5B00E250394BD8382350D1
:1036C00004302250C4225200A350C623E4205B00E1
:1036D000E1500433334AE1503349344BD16034492B
:1036E000800019503349E938FF3819503249043005
:1036F000195032493248D16132491163324951631C
:103700001900F4310860CE20304940001160304982
:10371000195019002F48F83108602F49D1658221CE
:103720002E4A89005A501A002D490832D1671A00D2
:103730002C49B432116088212B4A89005A501A0052
:103740002A49883211602A4ADA6407F061FD0120B3
:1037500007F0AEFFF8BDC0460004FF1F2C64FF1F3A
:10376000106FFF1F2444FF1F4A0AFF1F3A07000083
:1037700080C3C9019A020000DC0500006A1800003D
:1037800050C3000088130000F009FF1F204E000006
:103790006509FF1F68100000C409000040420F00C7
:1037A00010270000FC00FF1FC11BFF1F0000FF1FB0
:1037B000152CFF1FA52FFF1F3D2EFF1F811FFF1F71
:1037C0007126FF1F9D1FFF1F4921FF1F0D1FFF1F98
:1037D0009528FF1F7D29FF1FD918FF1FA127FF1F55
:1037E000C524FF1FD124FF1F0D1EFF1FC51EFF1F75
:1037F000851DFF1F0223F0B50124634D634E2B701E
:10380000634B91B01C70634F039333680021082011
:10381000BB7006F0F9FB082006F0F0FA002398428E
:1038200005D0BA78552A02D0332A00D09FE0336001
:10383000042006F063FD07F0DBFEFFF75DFE07F0F6
:10384000FFFE1F2201240021534B10AE1A70534B70
:103850001C70534B1970534B19689143163A0A4325
:103860001A60602219689143403A0A431A6007F0CF
:1038700007FD07F0D5FEC120FF214B4B80001A58F1
:103880008A431A50C522920098588843BF39014391
:1038900099509858454908408021C901014380202A
:1038A00099509958C0050902090A0143995080218D
:1038B0003F48490107F0D4FE032322003D4901940B
:1038C00000933D4807F024FD2C223C4905A807F051
:1038D0007FFF05AC61782078023406F0AFFAA6428B
:1038E000F8D1374C0121002006F0BCFB0920012152
:1038F00006F0B8FB2268334B03201A40A023DB02FA
:1039000013432360802322689B04134323602268AF
:103910002D4B1A4080239B03134323602B4A2C4BCF
:10392000934200D8012007F01BFD07F081FE8023A1
:103930002268DB0413432360287807F0F9FD039B1A
:103940001878C0B207F014FF07F0C2FC2149042028
:1039500007F046FE06F09EFC00F0A8F800F0C0FD5F
:1039600000F068FE00F00CFA002011B0F0BD0093EA
:103970002100184A042007F0A3FE8023DB059C6287
:10398000FFF764FD54E7C0464A0AFF1F34F00040C9
:103990002444FF1FC061FF1F480AFF1F490AFF1F81
:1039A000680AFF1FBCF0004000E100E0FF00FFFFDD
:1039B0002844FF1FAC56FF1F2854FF1F60B800119A
:1039C00014F00040FF7FF8FFFFFF9FFF0080FF1F04
:1039D000106FFF1F3B00010870B500252549264ADE
:1039E00026484D6308CA1B051B0DED188242F9D10C
:1039F00000268022224B92058B630921214B224C09
:103A00001E62224B1120DA67214BDA688A43DA60A2
:103A10009A6820490A409A60266007F0F1FC11205C
:103A200007F06EFD8022636C93436364EE24E40030
:103A30006C43194A200C0400642390420AD8FA22ED
:103A40003300D200904205D9144B0A21C01807F068
:103A500027FDC3B2124A11201372D48007F060FC14
:103A6000104B1B78002B04D10F4B1021187807F056
:103A700027FD70BD00000540880505400006054093
:103A8000FF01000000F000400038004004E100E0C9
:103A90003CF00040FFDFFFFFB70B000030F8FFFFF6
:103AA000A861FF1FE263FF1FE061FF1F002210B546
:103AB0001100112007F004FC10BD0000F8B5002330
:103AC0000926374F374C3B62E3681120B343E3606C
:103AD00007F016FD112007F093FC112007F008FCF9
:103AE0004023226880251343236080236268DB0221
:103AF00013436360A3682C4A2B43A360A36802218D
:103B00001340A3608023A2689B0113431022A3608B
:103B1000236C072093432364236C0F3A13432364DD
:103B200080235B003B62226B204B1A402263626B56
:103B30001A406263A26B1A40A263E26B1340E36314
:103B4000E3681B4A1340E36006F078F9012107207F
:103B500006F088FA174B11205A6C15435D6407F084
:103B600017FEFD21144B154A89005A508023C720A7
:103B7000626B5B0313436363E36880003343E3607A
:103B80000F4B104A19581140802212020A431A5052
:103B9000802292051A6008220B4B5A63F8BDC0467A
:103BA00000F000403CF00040FFFFDFFFEFFFEFFFC1
:103BB000FFFF7FFF003800400000FF1FD9390011D0
:103BC00000E100E0FF00FFFF0000054030B503A862
:103BD00004880B20002C0ED14968074D08784978DD
:103BE000090201430A20A94205D1012120001980C0
:103BF000024B1B7A137030BD192A0000A861FF1F09
:103C0000F7B5150008AA16884A680F4F147852783D
:103C1000120222430A24BA4214D10122DBB20192D9
:103C200000962A0007F086FA041E0BD1074B1B688A
:103C3000002B07D068782A78000210434242504196
:103C4000013098472000FEBD022900002C61FF1FB3
:103C500030B5012503790400BFB02B4211D00A49C9
:103C6000408806F0D3FD28420BD0084B01A95B8D9C
:103C70004D800B80064B00221B7A60880B7103F08D
:103C8000A5FE3FB030BDC0462461FF1F6840FF1F46
:103C9000A861FF1F10B50549054806F06DFD042118
:103CA000044A054806F02AFD10BDC0462461FF1FE6
:103CB000FFFF00008CB800116840FF1F10B50248DC
:103CC00004F006FD10BDC046513C0011062310B59E
:103CD000837010330371443B43712A33837144333F
:103CE000C37100230222012103720E4B0270417046
:103CF0001C8881724472197A0273C1729A78427375
:103D0000DA7882730322C2731A7902745A79427480
:103D10000C2282749A79C274DB7903751123C37003
:103D2000152010BDA861FF1F10B5142007F0B8FCC6
:103D3000124B14220021186007F01AFB002007F034
:103D40001FFB012007F06CFA022007F091FC032012
:103D500003F062FF042005F077FF052003F0A0F9CF
:103D6000062003F06DFE072001F004FA082006F09B
:103D7000A5FC092000F0E6FF10BDC0463061FF1F22
:103D800007F02EFB012007F01BFC07F0E9FC000008
:103D9000094B10B50400984205D0012904D1200038
:103DA000064906F0E9FC10BD0229FCD1013904F0F6
:103DB0004DFC0028F3D0F6E7FEFF00005661FF1F20
:103DC00070B50D7A100004AA2C0016881022144039
:103DD000154220D1002E20D10A78022A18D14A6833
:103DE000517815780E4A09022943914205D00D4AAF
:103DF000914209D01C800A2404E014220A491A8046
:103E000007F0E6FC200070BD0C2208491A80F7E795
:103E10001C800124F6E70824F4E70B24F2E7C046EF
:103E2000F3FF0000F4FF0000B042FF1F6CB9001167
:103E300010B504000749084806F09EFC074804F046
:103E400087FB0020E40704D50721054A054806F052
:103E500055FC10BD5661FF1FFFFF0000913D001192
:103E6000D0B80011AC40FF1F00B50C4BBFB01A78A2
:103E70000B4902A800F098FC6B4680B2D88000285D
:103E800009D06A46074B01A91B889380064B002284
:103E9000188803F09BFD3FB000BDC0463461FF1F92
:103EA0003561FF1F0641FF1F1042FF1F00B50C4B7D
:103EB000BFB01A780B4902A801F0CEFC6B4680B265
:103EC000D880002809D06A46074B01A95B8D9380F2
:103ED000064B0022188803F079FD3FB000BDC046B4
:103EE0005E61FF1F5F61FF1FAC40FF1F1042FF1F9D
:103EF000F7B50E00377A1C0008AB11003D001A8898
:103F000020231D401F423CD13378022B3BD17368E4
:103F10001F785B781B023B431E4FBB4208D01E4FED
:103F2000BB4214D01D4DAB4221D00A252800FEBD56
:103F3000002A2AD1142C2AD82200F06807F048FC65
:103F4000174B1C70012CF1D9FFF7B0FFEEE7002AE8
:103F50001BD1202C1BD82200F06807F039FC114B34
:103F600004211C70104B187807F0AAFADEE7E3B2C0
:103F70000124009201940A00310007F0DBF80500EB
:103F8000D4E70825D2E70125D0E70B25CEE70D259C
:103F9000CCE7C046F3FF0000F4FF00000229000058
:103FA0005E61FF1F3461FF1FE061FF1F332310B507
:103FB000040003700A220749013007F009FC064B90
:103FC0000F201B681A0AE37222731A0C1B0E62730D
:103FD000A37310BDA861FF1FD061FF1F30B501257D
:103FE00003790400BFB02B4213D00B49408806F080
:103FF0000DFC28420DD06A46084B02A81B8893800E
:10400000FFF7D4FF6B46D8800022608801A903F037
:10401000DDFC3FB030BDC0465661FF1F0641FF1FAB
:1040200010B5024804F054FB10BDC046DD3F00113E
:1040300070B5160004AA148805AA15784A68507845
:10404000117800022A4A0843801805284BD807F047
:1040500047FA03131E29343F0720042C0BD80522EE
:10406000121BAA4200D92A0022491A8030000919DD
:1040700007F0AEFB002070BD0720112CFBD81222E8
:10408000121BAA4200D92A001B491A80EEE707201A
:104090000E2CF0D80F22121BAA4200D92A00174971
:1040A0001A80E3E70720032CE5D80422121BAA425A
:1040B00000D92A0012491A80D8E70720032CDAD841
:1040C0000422121BAA4200D92A000E491A80CDE709
:1040D0000720032CCFD80422121BAA4200D92A00A1
:1040E00009491A80C2E700220A201A80C3E7C046A5
:1040F000DCD5FFFF1BB900117C61FF1F0BB900115C
:1041000006B9001101B90011FCB8001110B50D215C
:10411000024A034806F0F2FA10BDC046F0B800119A
:104120001C41FF1FF0B50024274E85B03000B4714C
:1041300000F0E2F8254D264BEA89297C9A422FD1DE
:104140000423300003AA00F057F90400300000F007
:1041500011F90123B371002C34D16B4699892B6876
:10416000C9BA4B4329891B4A1B145B1853806B4601
:10417000D9896B6849BA89B24B4369891B0C5B18B2
:104180001548191C1BB2834200DD011C0B0400D52D
:1041900000211388918001331380200005B0F0BD09
:1041A0000227220003AB3000009700F0F7F80E233F
:1041B0000400297C0122300000976B4400F0EEF8E7
:1041C0000443C3E71C00E8E7F441FF1F9061FF1FB1
:1041D00083050000A861FF1F0F27000073B5234E61
:1041E000300000F089F8224D07236A463000297C10
:1041F00000F002F904003000002C33D16B461B782C
:104200007F2B2FD800F0B6F86B46D878F023020445
:104210001B031A406B469B8816495BBA9BB21A4334
:104220002B68000953432A891B0C9B184B806B4653
:104230005A789B7812031B011A436B68024353435D
:104240006A891B0C9B180C481A1C1BB2834200DDA8
:10425000021C130400D500220B888A8001330B80D6
:10426000200076BD00F086F80124F9E7F441FF1F35
:104270009061FF1FA861FF1F0F27000070B5114C50
:10428000237C002B0FD0382B0ED10F4D280000F0CF
:1042900033F8CC23AC222800217C9B0100F0F4F8F9
:1042A000280000F067F870BD084BE2899A42FAD105
:1042B000054D280000F020F800222800217C00F0A5
:1042C000C5F8EDE79061FF1FF441FF1F8305000073
:1042D00010B5084B1A7C002A09D05B69002B06D068
:1042E0009847041E01D0FEF78BFE200010BD01246C
:1042F000F9E7C0469061FF1F70B5C17905000C0059
:10430000631E9C411A4BE402E41849000460C9B2E0
:10431000007905F0DDFEE979687949000131C9B21B
:1043200005F0D6FEE8790930C0B206F0E1FF0023BF
:10433000E36661332360AA795B3B002A0ED02268D2
:104340009A43023B134323600A23E361073323624A
:1043500000232363A3630133E36370BD22689A43A0
:10436000022313432360462363610633A361EFE70F
:104370000050004070B5002504000368DD66C07978
:104380000930C0B207F0BCF82900207905F03CFEE6
:104390002900607905F038FE70BD0000F8B51E00F8
:1043A00006AB1D78002304681700E366616007F020
:1043B0006FF901238022E3662B0027615200013B45
:1043C00008D206F045FF08200A4A1168002D03D1E3
:1043D0002800F8BD2261F2E7236F034203D023696E
:1043E000013D3370013613685B1A032BEED90125AA
:1043F000EEE7C0466008FF1F70B51C00002305688B
:104400001600EB66696007F043F901238022EB6632
:1044100023005200013B08D206F01AFF08200A4A86
:104420001168002C03D1200070BD2A61F2E72B6FC8
:10443000034203D02B69013C3370013613685B1AC9
:10444000032BEED90124EEE76008FF1F002370B5AF
:1044500004681500E366616007F01AF90123E3665A
:10446000256106F0F5FE8020064A80001168636B26
:10447000034205D113685B1A032BF8D9012070BDE4
:104480000020FCE76008FF1F70B51D0000230468D2
:104490001600E366616007F0FBF80123E36626611E
:1044A0000F33626B1A42FCD02B0A23611023626B1C
:1044B0001A42FCD0EDB2256106F0CAFE8020074A00
:1044C00080001168636B034205D113685B1A032BEC
:1044D000F8D9012070BD0020FCE7C0466008FF1F2E
:1044E00010B5084CE368002B08D18022064B52021D
:1044F0001B689B186360054B1B68236007F088F8F6
:10450000A06010BDD061FF1FC8F00040CCF000409B
:1045100070B5184A936A916A9942FBD116498A6824
:104520009A421FD39A1A8B60144B0126186893B2D3
:10453000D202D20E4343424300204C681B0A1B198F
:1045400012029B180E4C0A684B60551CA3420CD8F3
:10455000002801D04B600A600A4A136008680A4BC1
:10456000186070BD581E821ADDE7084A30009B189B
:104570002A00EAE700F00040D061FF1F140AFF1F85
:1045800040420F00C8F00040CCF00040C0BDF0FF3A
:1045900070B51F4C23793F2B01D93F2323711D4B4D
:1045A00022791A701878C0B207F0C2F818231A4995
:1045B0001A4A0B801A4913800B805380A37919493A
:1045C00080200B800C21938001334B43164D191C26
:1045D0000001834200D9011C2980D1806379002B1E
:1045E00011D101336371237A012B01D80223237285
:1045F0006279237A0D4853430A21584306F050FF4D
:104600000B4D286070BDA02BEDD9A023EAE7C04672
:10461000C461FF1F480AFF1F0E42FF1FD043FF1F48
:104620000C42FF1F0A42FF1F0842FF1F71020000D9
:10463000B461FF1FF8B514210020FEF7CFFE114C26
:10464000011E114D09D10C22104BC1CBC1C4280051
:1046500006F08EFEFFF79CFFF8BD0C2220000C49EF
:10466000FEF790FE0C2802D0084B43CB43C40C222B
:1046700028000849FEF786FE0C28EBD00C2200210A
:10468000E5E7C046C461FF1F9061FF1F60B90011DC
:10469000FC0C0000F50C0000F0B51D4C8022A54478
:1046A0000400882069465201400506F0A9FD9022C9
:1046B00012016A441300200032C832C316C816C360
:1046C0008023144C144FA6689B033343A3603B60C4
:1046D00006F096FF8823A0685B05C01806F0A8FEC8
:1046E0000025882329008022A0685B05C018401996
:1046F0006944520006F0CCFE80230135FF355B0192
:104700009D42EED1A6603E60044B9D44F0BDC04684
:10471000FCEFFFFF4043FF1F9808FF1F041000003D
:10472000F0B5040087B0002825D0684606F0E8FD03
:104730001B4C022806D106226946200006F020FF05
:10474000002816D06946002301250F262F00E25CC1
:10475000013310091030874038002F003240974055
:104760003A0002434A610439062BEFD16846FFF74D
:1047700093FF07B0F0BD182269460A4806F040FDD5
:104780006A46A300D358013305D01822FF2168469A
:1047900006F0EEFDEAE70134062CF1D1E9E7C04668
:1047A0006509FF1F00090011F0B5002504000E0087
:1047B00085B0AA4200D183E04B1C087801934B7866
:1047C0008978377909021943F3783F061B040B43B4
:1047D0001F43039720706570252800D193E033D8DC
:1047E000112813D806F0E4FE66000D010D010D013D
:1047F0000D01A700B500AE000D010D010D010D0169
:104800000D010D010D010D01E7000701232800D165
:10481000C0E0DB2800D016E1042A00D8A9E010256A
:10482000052A05D0551F2A003800711D06F0D0FF5B
:1048300005223100200006F0CBFF2A003900601D60
:1048400006F0C6FF05353BE0562856D010D8332871
:1048500000D19AE0552836D02628DAD1894B290094
:10486000132218001D0006F083FDFEF7C9FB59E076
:10487000712800D174E0722800D17DE0DC28C8D115
:10488000022A00D875E07378BFB26370B378A37062
:10489000032A05D0033A390092B2F01CFEF7ACFCB3
:1048A00010223900E01CFEF76DFDC51C002807DA58
:1048B00060705CE00C222000734906F089FF0C2533
:1048C000280005B0F0BD013A704D0C2A13D8002A1B
:1048D0000AD02800019906F07BFFFFF759FE0C2251
:1048E00028006B49FEF788FC29000C22601C06F0AA
:1048F0006FFF0D25E4E70C22EBE7644D654B2A00C2
:1049000043CB43C2E9E7013A5E4D0C2A11D8002A95
:1049100008D00199280006F05BFF0C2228005E49B0
:10492000FEF76AFC29001322601C06F051FF1425D3
:10493000C6E70C22EDE705225849601C06F048FF47
:104940000625BDE712225649601C06F041FF1325DB
:10495000B6E708225349601C06F03AFF0925AFE785
:104960007178F02905D8504B188801F0D1FB022549
:10497000A6E7FF236370FAE74C4B012A03D0727855
:104980005A706270F3E75B78F4E72000FFF70EFBE4
:10499000050095E7042A04D9454D2F6006F038FE3E
:1049A000A860FFF7B5FD0422039003A9601C06F080
:1049B0000FFF052584E73F4D062A15D9062228005A
:1049C000019906F0DDFD00280ED00622019928008D
:1049D00006F0FEFE062238492800FEF70DFC0123F2
:1049E000324A51780B43537029000622601C06F0AE
:1049F000EFFE072564E7012ABBD07078FFF790FE31
:104A0000B5E7012800D004E7931E2C4F1A2B04D8D9
:104A10007378002B09D100F009F9294B39001D7872
:104A2000601C6A1E06F0D4FE4AE7551E2A00019952
:104A3000380006F0CDFE2349AAB23800FEF7DCFBB1
:104A400000F02AF9E9E7DA2893D1042A91D9082A53
:104A500015D9B37972791B021343F27912041A4300
:104A6000337A1B0613433B603B680522310020006C
:104A7000039306F0ADFE0422601D03A96CE7FE233C
:104A80006370F1E79061FF1F6CB90011C461FF1FF3
:104A9000FC0C000060B90011F50C00009C61FF1FC8
:104AA0007C61FF1F4443FF1F1042FF1FC061FF1FB7
:104AB000D061FF1F6509FF1FADAC0000C163FF1F80
:104AC000BF63FF1FAEDE000070470000020010B59C
:104AD000094B0A32094C92B2DA815A8298811882C3
:104AE000207802F07BF90422054B012120781A700E
:104AF00006F0E6FC10BDC046CE42FF1F0A64FF1F51
:104B00000964FF1F013870B5042809D806F0E8FCD5
:104B10000309230812001E4B0221187806F0D0FC6E
:104B200070BD1B4B0821187806F07AFE0022194B45
:104B30001A72F5E780220024164B154D52001A8197
:104B4000082128781A68DC7206F09AFC210028787F
:104B500006F006FDE4E70E4B0821187806F060FE2B
:104B60000D48FFF7B3F80D4B0D4A9B7993800D4A22
:104B700013800022074BDA720132FF321A810A4B8E
:104B80005B78002BCCD0094A136006F031FEC7E7F2
:104B9000E061FF1FB461FF1F1942FF1FC461FF1FC7
:104BA000D043FF1F0A42FF1FC061FF1F34F00040C7
:104BB00010B5002905D1082803D10131013005F0D5
:104BC00051FA10BD10B501290FD108280DD10021CF
:104BD000013005F047FA054B1B78002B05D0262243
:104BE000034B04485A72FFF771FF10BDE263FF1FC9
:104BF000B461FF1FC40900000300F0B50A4D8E1810
:104C0000B14202D152008018F0BD0C782F682409FF
:104C10003C5D0F271C700C7801313C402F683C5DD7
:104C20005C700233ECE7C0460442FF1F0E22114BBA
:104C300010B51A700D23104C10492370093A043B2B
:104C40000F48637006F0C4FD2D2301220D490E4864
:104C5000E371FFF7D1FF01220C49FFF7CDFF0122DD
:104C60000B49FFF7C9FF00220A491000FEF7C4FAFA
:104C700010BDC046DE63FF1FBF63FF1F1BB90011DD
:104C8000C163FF1F6709FF1FC763FF1F6609FF1F7F
:104C90006509FF1FAEDE000070B5124C1322200024
:104CA0001149FEF76FFB114D002817DDAB78002B83
:104CB00014D0431C2B7009236B7000230019037060
:104CC000287829000130C0B206F002FC29782200C1
:104CD0000139C9B2002005F02FFC70BDFFF7A6FF17
:104CE000EEE7C046C163FF1FAEDE0000BF63FF1FDB
:104CF00010B5114B1A781870002A0ED000280BD16D
:104D00000E4B1A78062A07D85423D340DB0703D565
:104D10000B4B187802F062F810BD0028FCD0074B4E
:104D20001B78012B02D0033B022BF5D8044B012149
:104D3000187806F0C5FBEFE7E263FF1F0964FF1F69
:104D40000A64FF1F70B5504E504A51493070082018
:104D500005F07EFA0121092005F084F9092005F00B
:104D600065FA0121002005F07DF9002005F05EFACA
:104D7000FEF746F906F00CFC032246494648FFF7C9
:104D80003BFF2D24030004221C7044490130FFF72F
:104D900033FF30230470424D424C437083702E3BEE
:104DA000062220004049EB87FEF7ECFA062813D0D4
:104DB000200006F0A5FA022809D00321200006F001
:104DC000C7FC8D23E3706E3B237119336371062298
:104DD00020003549FEF710FA344B1B68FC335C6445
:104DE000FFF75AFF0020FFF783FF314C314A0121C2
:104DF000314B1278207801F0B3FF304A304B1278F3
:104E00000021207801F0ACFF01222E4B1A702E4BAE
:104E10009B78552B31D12D4B3B325A722C4B2D4A5E
:104E2000AB81EA812B826A822021307806F0C0FAB9
:104E30000120404205F0CCFB0120404205F068FC17
:104E4000FFF764F9FEF726FF00F09EFC01204042C8
:104E5000FEF7EEFF012006F09BFAF02001F03CF98E
:104E60000121307806F02CFB307802F013F91A4853
:104E700006F086FCFEF722FE70BD6422174B5B79BC
:104E800053431A000A32CBE7E061FF1FB14B001118
:104E9000C54B00114443FF1F7C61FF1F9C61FF1F36
:104EA000CE42FF1F6509FF1FADAC00002C64FF1F41
:104EB0000A64FF1F3842FF1F1942FF1FDE63FF1FF6
:104EC000BF63FF1FB063FF1FC061FF1FB461FF1FFF
:104ED000C4090000CE090000E261FF1FC461FF1F8A
:104EE000F8B50A0020230D001A40194251D0544B46
:104EF0001B78002B3CD0FFF70BFB524B524C534E10
:104F000099686268737A8A1ADB039A4202D36160F5
:104F1000FEF7D4FD327A217A531EDBB299422AD1B0
:104F2000FFF7ACF9637A002B1FD0013BDBB2637251
:104F3000002B1AD1464B9B78552B01D106F058FC1B
:104F4000E37A002B0CD00023424A434FE3721388CC
:104F5000380001331380FEF7B9FE390006F0A0F9DE
:104F6000642370795843FFF7B1FD237A013323722C
:104F700020206840F8BD9142D4D300232372FFF76C
:104F8000A7F9354F3800FEF7A1FE390006F088F981
:104F9000C8E70BB2002B0ADA304B187806F070FB2A
:104FA000002801D006F0CCFB80200002E1E70224BB
:104FB000214206D0244B01201A72FFF799FE2000EF
:104FC000D7E70B071BD5FFF7A3FA1E4B1E491F4C53
:104FD00098684A68637A821ADB039A4202D348606F
:104FE000FEF76CFDFFF774F9FFF748F900F0E6FBF8
:104FF0002368DB0701D5FFF713F80820B9E7102471
:105000000E002640214206D00D4B1B78002BD6D136
:10501000FEF754FED3E70124214209D0104800F0E6
:105020006DF806F00DFC3100092005F01BF8C6E70D
:1050300004240800204021429CD0FEF715FFBEE763
:10504000E263FF1FD061FF1FB461FF1FC461FF1F38
:10505000C061FF1FA861FF1F1942FF1FE061FF1F12
:10506000FC41FF1FF0B51B4B1B4F1B883A88040007
:105070001A4E1B4D85B09A420DD832889A420AD3F7
:10508000184B1A882B889A4205D1174A174B128859
:105090001B889A421BD0052001F074F83B8802AAB5
:1050A00013803388019053802B88114D93800F4BD0
:1050B00002A91B88D3800F4B2A78188802F090FD34
:1050C0000D4B08212878019A1C7006F0B9F805B03C
:1050D000F0BDC046AE63FF1F0E42FF1F0C42FF1F14
:1050E0000A42FF1FAC63FF1FAA63FF1F0842FF1F96
:1050F0000A64FF1F1042FF1FA863FF1F13B50C4B6C
:105100001C78002C11D1002801D00A4B18600A4AE3
:105110000A4B11780A4A10780A4A01920A4A009208
:10512000002205F001F9200016BD1124FBE7C0465E
:105130000964FF1FA463FF1F0864FF1FF863FF1FBC
:105140000A64FF1FE463FF1FE863FF1F10B5064BEF
:1051500012201B78052B06D1044B13221988044B0F
:10516000187801F0EBF910BD0964FF1F1042FF1F12
:105170000A64FF1F10B500240122114B524218701F
:10518000104B1C70104B1A8001F084FF04220F4B4F
:1051900021001A700E480C3206F062F8102221002D
:1051A0000C4806F05DF807220B4B1C600B4B1C7083
:1051B0000B4B1C700B4B1A700B4B1C7010BDC04678
:1051C0000A64FF1F0964FF1F1042FF1F0864FF1FCE
:1051D000F863FF1FE863FF1FE463FF1FBE63FF1F49
:1051E000BD63FF1F1242FF1FBC63FF1FF8B5174CC2
:1051F0000600257806A814240078052D23D1B41FB5
:10520000134FA5B21824BD421DD88D1FADB2BD42AB
:1052100019D8FA256D00AA4215D21D000D4F0A3D7E
:10522000ADB2BD420FD80C4C26800C4C21800C49ED
:1052300000240A800B4A1380FFF714FF0A4B042155
:10524000187806F0EDFA2000F8BDC0460964FF1F8B
:10525000790C0000750C00000E42FF1F0C42FF1F6E
:105260000A42FF1F0842FF1F0A64FF1FF0B50BB27E
:105270000D0089B0002B00DB70E1A44E307806F001
:10528000FFF9041E50D00378A22B00D122E1D02BCD
:105290001AD0912B45D143780E2B42D19C4B82885A
:1052A0009A423ED19B4A83681278052A39D103205D
:1052B00018567F2835D0984B1B68002B31D05B687F
:1052C000002B2ED098472CE08078072829D806F0AC
:1052D00007F90428183F3F74A8D86378002B0CD135
:1052E00001218C4B19708D4B1A78002A5BD08C4BA6
:1052F000307801F035FD002855D00722854B1A7013
:1053000051E061780029F8D1E378002B11D0854A6B
:10531000854B1278307801F023FD60706378002BA4
:10532000EBD1200006F00CFA80200002684009B0A2
:10533000F0BD784B1B78022BF3D00121307806F0BA
:1053400067FA0028EAD10121307806F0B9F8E5E7DC
:105350006378002BD1D16F4F032807D13B78052B01
:1053600002D101333B701EE00223FBE76F4B1A882A
:105370006F4B0293002A0BD01B78002B03D0012126
:10538000307805F05DFF3B78062B04D1013BE9E75F
:10539000029B1A70F7E7042B41D10121029B307860
:1053A000197006F08DF85C4B1B68002BB9D01B6898
:1053B000002BB6D0574A107884E76378554F002BFE
:1053C00027D10622211D5B4806F002FA62895A4B5A
:1053D0005A491A80A2895A4B1A80E3890B80052109
:1053E000397058490A80584A1380228A574B1A80CC
:1053F000574B1B78012B09D11F2000F0C3FEFA2266
:10540000920042430421307805F01AFF0022484BF5
:1054100075E7312B00D070E70022454B1A7003234B
:10542000A0E706220021434805F01AFF0023454A61
:1054300004211380444A30781380444A138006F0D4
:10544000EFF90821307806F0EBF9A379083B5A42CE
:105450005341304A03331370304B1B78002B06D076
:10546000334B30781A78002A06D001F0B7FC0122BD
:10547000314B52421A8096E70121197006F020F84C
:10548000F5E70821307806F0CBF96378002B00D0DF
:1054900047E72C4B2D4F0293E388029A0421138097
:1054A000294B307803932389039A138063893B80C7
:1054B00006F0AEF9002800D033E7264B1B68002B1E
:1054C00000D12EE7039902983A88098800881B6862
:1054D000984726E74379132B00D022E70389012B55
:1054E0000AD11D4B1B78022B06D10821307806F01B
:1054F00097F9FFF72BFE14E7052000F043FE082183
:105500000200307805F09CFE0BE7C0460A64FF1FDE
:10551000051400000964FF1FA463FF1F3842FF1F2A
:105520001942FF1FDE63FF1FBF63FF1FE063FF1F02
:10553000E263FF1FB163FF1F1042FF1FB863FF1F2D
:10554000BA63FF1FAE63FF1FAC63FF1FAA63FF1F99
:10555000B063FF1FA063FF1FA863FF1F8020C0016F
:10556000014200D0E2E6CB0731D5324B1B78002B4D
:105570001DD0314E05AC3378052B1AD1023B237078
:105580002E4B21001B7823722D4B1B7863722D4B01
:10559000187801F089FB002809D007202A4B3070C9
:1055A0001B68002B03D01B68002B00D098470120FC
:1055B000BCE60E20254B06221B7825492370254B7F
:1055C0001B78637002ABC01806F002F9D8E702231B
:1055D00008001840194209D0174B1B78052B03D13E
:1055E0001D4B188805F044FE02209FE6042421424A
:1055F00003D0FFF737FD200098E608230800184085
:10560000194200D193E6154B1C78012C03D0022CD3
:105610000DD008208AE6124B124A134913481B8802
:105620001288098800880094FFF7E0FDF1E7FFF792
:105630008DFDEEE7E263FF1F0964FF1F1242FF1FAB
:10564000BC63FF1F0A64FF1FA463FF1FBE63FF1F2D
:105650001342FF1FBD63FF1F1042FF1FA863FF1F00
:105660000842FF1F0A42FF1F0C42FF1F0E42FF1F8E
:1056700010B502A804880B20002C10D149680878C6
:105680004978090201430C48814209D1022119805D
:105690000A4B59881170DB7800205BB2537010BD43
:1056A000074C0A20A142FAD102211980034B9988A4
:1056B00011705B79F0E7C0466E2A0000A861FF1FF9
:1056C0006F2A0000F7B5150008AA16884A680F4F20
:1056D00014785278120222430A24BA4214D10122C9
:1056E000DBB2019200962A0005F024FD041E0BD1C6
:1056F000074B1B68002B07D068782A7800021043FC
:1057000042425041013098472000FEBD022900006E
:105710001C64FF1F30B5012503790400BFB02B4284
:1057200025D01449408805F071F828420CD0124B5E
:1057300001A95B8D00220B8002234B800F4B5B88FD
:105740008B80608802F042F90D49608805F05EF8B0
:10575000C0070CD50B4B01A91B8800220B8002232C
:105760004B80064B9B888B80608802F02FF93FB0FE
:1057700030BDC0461464FF1F3C42FF1FA861FF1FDD
:105780000C64FF1F9642FF1F10B5074C074920000D
:1057900004F0F2FF2000064904F0EEFF0721054A5D
:1057A000054804F0ABFF10BDFFFF00001464FF1FAD
:1057B0000C64FF1F8CB900113C42FF1F10B502485A
:1057C00002F086FF10BDC046155700110200F0B56B
:1057D00001270A480A4E51188B1A002B00DCF0BD35
:1057E000082415784308684038404000805B013C3D
:1057F00058406D08002CF5D10132EDE7FFFF0000A5
:10580000A6B90011F0B500250F269D4200DBF0BDC2
:105810004C5D070944403440A400A058013578404D
:10582000F3E70000F0B589B06A460D000B000F27C2
:10583000110010351C780133260024093E401670F3
:1058400054700232AB42F5D12023024AFFF7DAFF4F
:1058500009B0F0BDACB90011F0B54E780B7889B045
:1058600036020C00170001901E43012A61D9954BA6
:105870009E4200D877E001339E421CD1062A17D100
:10588000CA788B7812021A430B791B0413434A79A6
:1058900012061A438C4B5A6100221A705A808B4AA6
:1058A0005A608B4A9A608B4ADA60002009B0F0BDDA
:1058B00088225205EEE7884B9E423CD182498B7884
:1058C000002B00D0F6E00C2A31D10F22A3789343AD
:1058D000E27812021343227912041343627912060A
:1058E00013434B60E279A07912020243207A00044C
:1058F0001043627A12060243CA60E27AA07A120268
:10590000024376484A81834208D804236E49142210
:1059100001980B7005F05CFF1420C7E71201D21844
:1059200089235B059A42F0D801238B70BDE7022AD8
:10593000FAD00523EAE76A4A01239642E6D1FFF747
:1059400005FC052F0CD9E378A2781B0213432279BA
:1059500012041A4363791B061343624A03931360CC
:1059600005F046FFA1E7584D2B78002B9DD1AB7871
:10597000002B00D1A0E02B8901339BB20093B342EE
:1059800000D091E0132AD4D9CF7C8B7C3F02122126
:1059900020001F43FFF71AFF874200D08EE0002E41
:1059A0003DD1E378A2781B0213432279E9681204FF
:1059B0001A4363791B06134303930A228B4212D1C5
:1059C000FF23A370E370237163716B89002B09D1EE
:1059D000E37B227C1B0212041343A27B13431B09AB
:1059E00001336B8100226B89002B8ED0002A67D196
:1059F000686837013818000B6B6900030390984200
:105A000005D9686105F014FDEB780133EB70686827
:105A10001022A11C381805F03BFD2E8145E76F8947
:105A2000009A7B1E9BB293423AD1E278A37812028D
:105A30001A43237905A81B04134362796C68120684
:105A40001A43EB6800920392211D0C22049305F087
:105A5000BFFE0120260004A940421036FFF7E2FEF7
:105A6000013F012F17D1009A0B232861824200D0F9
:105A70004CE704221C49200005F00AFD042203A97A
:105A8000686805F0BDFBE968039AFF23914200D1E5
:105A90003CE7F73B3AE73100FFF7C4FE1036DFE79B
:105AA0000923B742A4D831E7009BB34200D9FCE6F2
:105AB00007232BE7022329E7032327E7062325E70C
:105AC0000A2323E7FFFE0000B042FF1F0000011180
:105AD000FFFF00005048593601FF0000FFFF001192
:105AE00002FF000034F00040BC42FF1F10B5034C21
:105AF0000B000122210000F06BFA10BDAD5C00111B
:105B00000B8870B506000D000224162B11D92B004E
:105B10000322094900F05CFA041E0AD1074B2A88C7
:105B20001B88191C934200D9111C300089B200F067
:105B3000EFFA200070BDC046D95C00114664FF1F1B
:105B400010B54A780400013A0B000220012A07D858
:105B50000A78002A04D005222000024900F038FA11
:105B600010BDC046075D00110A7810B50B00040097
:105B70000220002A04D007222000024900F028FA5F
:105B800010BDC046B35D00110A7810B50B000400CB
:105B90000220002A04D009222000024900F018FA4D
:105BA00010BDC046195E001110B5034C0B000B224E
:105BB000210000F00DFA10BD495E001110B5034C34
:105BC0000B000D22210000F003FA10BDBB5E001196
:105BD00010B5034C0B000F22210000F0F9F910BDA5
:105BE000155F00110A7810B50B0004000220002A8E
:105BF00004D011222000024900F0EAF910BDC0468D
:105C0000255F0011002310B51322190000F0E0F900
:105C100010BD000010B5034C0B001722210000F04E
:105C2000D7F910BD775F0011002310B519221900B4
:105C300000F0CEF910BD000010B5034C0B001B2284
:105C4000210000F0C5F910BDB15F0011F7B58489DE
:105C50000D0006000121002C22D000238268D356BB
:105C60001778002B1EDA0C2C1AD90C3CA4B213198D
:105C700040880093230002F086FE431E98410130C5
:105C80007B06DB0F6B703F23013C1F40A4B22870E2
:105C9000AF70AC80002C07D0B3680133AB6000213B
:105CA0000800FEBD0020EBE7AC60F8E70B7803705E
:105CB0004B8843704B881B0A83700B79C370042098
:105CC00070470420022B06D10020537811781B0264
:105CD000009A0B43138070470B8803700B881B0AD4
:105CE0004370022070470420009983420AD1537800
:105CF00010781B0203430B80D37890781B02034378
:105D000000204B807047F8B50D004B78012400212E
:105D1000461C03702B788B4201D82000F8BD6B78AD
:105D2000B01C4F1C012B10D1890069184B8802222E
:105D300033704B88B9001B0A7370691805F078FA44
:105D400004360434A4B2F9B2E4E7122359436B18C1
:105D50005A88043132705B8810221B0A73706918EC
:105D600005F066FA12361234ECE770B5049D1400A3
:105D70001E00052B01D8042070BD637812781B0229
:105D800013432B80E378A2781B02134302226B801B
:105D90002A71211D681D063E05F04AFAB2B22A8119
:105DA000E92AE8D82800A11D0A3005F041FA0020B0
:105DB000E2E7002310B50A789A4201D8900010BD9E
:105DC0009A008A185488013304705488DBB2240A7C
:105DD0004470948884709288120AC2700430EAE792
:105DE00010B51100029C062B04D004201022142BA5
:105DF00001D010BD022222714B7808781B020343A8
:105E00002380CB7888781B02034363800431601DB4
:105E100005F00EFA0020ECE710B50C788B78043111
:105E20005C43E4B203702200013005F001FA601C0B
:105E300010BD0420022B06D10020537811781B02DC
:105E4000009A0B431380704710B50C000A8802318A
:105E500005F0EEF9208810BD70B504000D0004981F
:105E60001100012B01D8042070BD1678527812025F
:105E7000324302800200F13255701470E125002C8B
:105E800000D10C35023B9AB24280AA42EBD80231D3
:105E9000043005F0CDF90020E6E7042000998342A4
:105EA0000AD1537810781B0203430B80D378907883
:105EB0001B02034300204B80704710B50C000A887A
:105EC000023105F0B5F9208810BD000070B5012140
:105ED0001E000420049C0E400B4218D1CB40DDB2C2
:105EE0008D4214D90A49DBB2098899420FD32300A5
:105EF000EE331D703300580011184978165C090202
:105F0000314301332152D9B28D42F4D8002070BD03
:105F1000C842FF1F10B50C000A88023105F088F94D
:105F2000208810BD10B50C788B7804315C43E4B246
:105F300003702200013005F07BF9601C10BD10B524
:105F400011000298032B01D8042010BD1478527858
:105F5000043B120222430280CA788C781202224348
:105F600042809AB28280EB2AEED80431063005F0E6
:105F70005FF90020E9E710B50C000B8803700B886F
:105F80001B0A43704B8883704B881B0AC3708A8836
:105F90000430063105F04CF9A088043080B210BD01
:105FA0000420012B03D100201378009A137070474E
:105FB00010B50C000B8803700B881B0A43704A88CD
:105FC0000230043105F034F96088023080B210BD2F
:105FD000F0B589B003931E4B029242000700D05ADD
:105FE000019102F020F81325061E2DD0029B0124FA
:105FF0000370019B002B04D00019039998470019E6
:1060000084B26B461B7A5BB2002B0FDA102138008A
:1060100002F01CFB1925002813D130003219E1B21F
:1060200002F066FC051E0CD10C34A4B2042304AAB1
:10603000380005A993800696948101F0AFFD051EF6
:1060400002D0300005F094FA280009B0F0BDC04637
:106050004464FF1F70B505000C0000280CD0002020
:10606000814209D010222000044905F0E1F8012006
:106070002B7823736B78637370BDC046ECB9001145
:10608000F0B506000D0017001C0085B002291BD0DA
:106090000020102907D1022B07D0102B03D115E0C7
:1060A0000020102C08D005B0F0BD69463800FFF77D
:1060B000D1FF2A0069460BE069463000FFF7CAFFAE
:1060C00022006946380004E0022BE9D12A00390099
:1060D000300005F00DFAE6E7031CF02800D9F023A4
:1060E000032008499AB2013A0B80D31703400649AE
:1060F0009B189B100B80D30F04499B185B100B80DF
:106100007047C046CC42FF1FCA42FF1FC842FF1F54
:10611000034B1B888B4202D3024B4000C152704795
:10612000CC42FF1F4464FF1F014B4000185A7047C8
:106130004464FF1F1722014B1A8070474464FF1FFD
:1061400070B505000E2005F0E3FA041E13D0D0232D
:10615000037000230622837007494570033005F061
:1061600067F8064B2100DA8A62811B7E2373044B99
:10617000187805F03DF970BD6064FF1F5064FF1F83
:106180001C43FF1F262803D8024B4000C05A70470B
:106190000148FCE7CE42FF1FFFFF000070B506007C
:1061A0000C00094D1C220021280005F059F8074B6E
:1061B0001E70074B1C7005F0F3F90123002801D075
:1061C000002312202B7070BD5064FF1F1C43FF1F63
:1061D0007164FF1F70B505000D4C0800E260A160FE
:1061E00010220021656005F07BF8012803D1102101
:1061F000A06802F058FD10220021280005F070F878
:10620000012803D11021606802F04DFD70BDC04629
:106210005064FF1F70B5041E05D1002903D006226B
:106220000D4805F005F80D4B1D78012D11D1002CFE
:1062300005D102221A7005F04BFA280070BD002229
:106240001A70074B1B78FF2BF7D02000FFF778FF61
:10625000F3E70025F1E7C0466064FF1F5064FF1FAD
:106260001C43FF1F030010B5002801D1002010BD02
:1062700000780B4A002803D15988D1821B79137604
:106280001378022BF2D10023984200D1033313700C
:10629000044B1B78FF2B01D0FFF752FF0120E6E7EC
:1062A0005064FF1F1C43FF1F002911D000280CD091
:1062B0004B79012803D140225242134303E03F228D
:1062C0001340032802D001204B7170474022F4E7AD
:1062D0000800FAE770B5094D0100287800280BD0B6
:1062E000074C0622200004F0A3FF21002878FFF7C6
:1062F000DBFF200005F02CF970BDC0467064FF1F65
:106300004A64FF1F00290AD0012808D13F224B7997
:106310009343C02B03D0403B5A425341981C7047D3
:1063200070B5174D06002B78FF2B15D00A2005F00D
:10633000EFF9041E10D0D0230370C83B8370114BBB
:1063400011491B784670C3700622043004F070FFB8
:106350002100287805F04CF80C4B1B78012B0DD14F
:106360000B4B1B68002B03D09B68002B00D0984779
:10637000084B04211878084A05F082F870BDC04621
:106380001C43FF1F7064FF1F4A64FF1F6C64FF1FE4
:106390009864FF1F9C64FF1F60EA0000014B98682F
:1063A0007047C0465064FF1F014BDB681868704798
:1063B0005064FF1F074B10B5DA6813680133136090
:1063C000054B1878FF2803D08021C90105F078F823
:1063D00010BDC0465064FF1F1C43FF1FF7B50E00E1
:1063E00002F0C8F8051E1CD00E4B06621F78002F65
:1063F00000D10778AB791020019305F089F9041ECC
:106400000FD0D0230380C73B8370019BE91DC3706D
:106410000622043004F00CFF21003800E66004F08E
:10642000E7FFF7BD1A43FF1F014B18787047C046BE
:106430007064FF1F054B002805D1054B1A78054BEA
:10644000002A00D1014B18007047C0466064FF1F4E
:106450007064FF1F4A64FF1F014B58687047C046B5
:106460005064FF1F024B1868431E9841C0B270472A
:106470007464FF1F421E03000120152A03D9FF3B4D
:106480005A425341D8B27047F0B51C0000230E00A9
:1064900085B0039002920B70029A934201D30020C0
:1064A00019E0E55C5A1CD2B2002DF8D002985119BF
:1064B0008142F4DC0233DFB2A35C18000193FFF7E2
:1064C000D9FF002807D0013D019A0399EBB2337040
:1064D0008A4202D1E01905B0F0BDDB19DBB2DBE77F
:1064E00010B50C0002F09EF803001220002B03D020
:1064F0002100588804F01CFF10BD000070B50E4D3F
:1065000084006359002B15D0186A002801D005F0CB
:10651000F7F82B59586A002801D005F0F1F82B59EB
:10652000986A002801D005F0EBF8285905F0E8F842
:1065300000232B5170BDC0468064FF1F1C4B70B5FB
:1065400004000E00150099420AD11A4B1B68002B5B
:1065500001D1122070BD1B68002BFAD09847F9E7D3
:10656000154B994215D1134B1B68002B0AD01B68A1
:10657000002B07D09847002804D1104B1C70104BFB
:106580001D70E7E729002000FFF7AAFF0028E1D1EE
:10659000F3E7080001F0EEFF0028DAD003780320CB
:1065A000A342D7D12900300004F0C2FED2E7C04692
:1065B000FEFF00007C64FF1FFFFF00007964FF1FE7
:1065C0007864FF1FF7B50400808801F0D3FF002531
:1065D000A84203D00578A08802F008F81C4E337852
:1065E000002B1FD0AB421DD11A4B28001978FFF7A2
:1065F00077FF002818D000233370A3790820A778EC
:10660000A688019305F084F8011E0DD0D0230370F5
:10661000CA3B8370019B477086808371280004F019
:10662000E7FE01E0002DE8D1A0880B4B8200D35893
:10663000002B01D0FFF762FF1721A088FFF768FD4C
:10664000A08801F027FDA08801F0FEFDF7BDC0463F
:106650007964FF1F7864FF1F8064FF1FF0B587B067
:106660001D000CAB1B88070001930DAB1B88142089
:1066700002930EAB1B88160003930FAB1B8800918F
:10668000049310AB1B88059305F042F8041E1AD042
:10669000D0230370CB3B47708370C670062229005D
:1066A0000430002D11D004F0C3FD019B2100638153
:1066B000029B0098A381039BE381049B2382059B9B
:1066C000A37404F095FE07B0F0BD04F0C9FDECE73B
:1066D000F7B5009308AB1B8807000C200D001600CF
:1066E000019305F015F8041E13D0280001F042FFB5
:1066F00000280FD00078D0232370C93BA370009BE3
:1067000021002381019B6770A580E680638104F0EE
:106710006FFEF7BD014B1878EDE7C0461C43FF1F25
:1067200013B5040064890389C2888188C078009405
:10673000FFF7CEFF13BD000010B5044C2068002801
:1067400003D004F0DDFF0023236010BD8464FF1F2D
:10675000A122F0B5818892004A43384B384F1B681C
:1067600004009B189D2292009B18827989B01A60C0
:106770003B68002B5FD01D78324B1B68002B04D088
:106780005B68002B01D000209847260008363100B6
:10679000E079FFF7B7FD237DE0710200E078049314
:1067A000638A29000393238A0293E3890193A388D0
:1067B00000933300FFF752FFE378002B0BD1E289FF
:1067C000A379A18802920196E27928000092012221
:1067D00001F0DAFEE0703B68002B20D0FFF7ACFF41
:1067E000194D287800281AD0184B1978FFF778FE31
:1067F000002814D02B78E67808200793A78804F0A7
:1068000087FF011E09D0D0230370CA3B46708370F6
:1068100087808671079804F0EBFD00232B70172109
:10682000A088FFF775FCA08801F034FCA08801F077
:106830000BFD09B0F0BD064B9DE7C0463409FF1FB4
:106840008464FF1F9864FF1F7964FF1F7864FF1F33
:106850001C43FF1FF8B5070008000E0001F08AFE78
:10686000041E18D02620FFF78DFC051E00D12578C8
:10687000062004F04DFF041E0DD00021062204F076
:10688000EFFCD0232370C23B21006770A370A68069
:10689000E8B204F0ADFDF8BDF0B585B001930AABE8
:1068A0001B78070002930BAB1B7808000D000092C9
:1068B000039301F05FFE061E22D0102004F028FF93
:1068C000041E1DD01022002104F0CAFC2620FFF770
:1068D00059FC002800D13078D0232370C13BA3702D
:1068E000009B21002372019B67706372029BA5804D
:1068F000A372039BC0B2E3720C9BE36004F078FDCB
:1069000005B0F0BDF7B50D00019001F033FE071E94
:1069100020D00E2004F0FCFE041E1BD02620FFF722
:1069200031FC061E00D13E78D0232380C53B0622D1
:10693000A370F91DE01C04F07BFC019B2A0063811D
:106940000123DD401A401D40210022736573F0B21F
:1069500004F04EFDF7BD0000F0B585B002901000C8
:106960000D0017000A9E039301F004FE041E31D0AF
:10697000029B002B2ED1039B02795B0724D51223A7
:1069800013430422002E08D10B99002905D10C993C
:10699000002902D10D9900291AD01A430D9B2271AA
:1069A000002B00D0C9E0002E00D1CFE0002D00D098
:1069B000CCE0606A002801D004F0A2FE1C21300067
:1069C00004F04EFD606205E002239A430E33D7E7E0
:1069D00093432371654BBA00D458002C00D1AAE030
:1069E000002E10D0236A002B03D11C2004F058FE87
:1069F00020625E4BBA00D358186A002803D01C22CC
:106A0000310004F015FC0C9B002B12D0574CBB003E
:106A10001D596B6A002B03D1162004F041FE6862F9
:106A2000BB00E358586A002803D016220C9904F0E2
:106A3000FFFB0D9B002B11D04C4DBC006659B36A77
:106A4000002B03D1142004F02BFEB0622B59986A5E
:106A5000002803D014220D9904F0EAFB380001F05D
:106A600089FD051E67D0414BBA00D358002B62D078
:106A70001A6A3420002A00D11C389A6A002A01D0F0
:106A8000143080B20B9A002A01D01C3080B25B6AAD
:106A9000002B01D0163080B204F03AFE041E4AD01A
:106AA0001822002104F0DCFB2620FFF76BFB01908D
:106AB000002801D12B780193D0232370029B200062
:106AC00063700A23294EA370039BBD00A371AB59C9
:106AD000A780196A1830002905D01C22A06004F094
:106AE000A7FB200034307359996A002907D00300AE
:106AF00014221433E060029304F09AFB02980B9B7B
:106B0000002B08D003001C221C330B992061029338
:106B100004F08EFB02987359596A002903D016229B
:106B2000606104F085FB6B462100187904F060FC7D
:106B30003800FFF7E3FC05B0F0BD10220D9B0D9966
:106B40001B69A018236204F073FB2CE70B9B002B3E
:106B500000D13FE7012D00D03CE7606A002801D05A
:106B600004F0CEFD1C210B982AE7C0468064FF1F6D
:106B700010B5044C2068002803D004F0C1FD0023A8
:106B8000236010BD7464FF1F0B4B07B51A68002A01
:106B900001D100200EBD6946531C01201278073137
:106BA000FFF772FC0028F4D002780123100018408F
:106BB0001A42EED0EEE7C0469064FF1FF0B51F4FBB
:106BC00001203B6887B0002B25D09B78059300F00F
:106BD000B3FB002821D00A20FFF7D4FA04000B20D1
:106BE000FFF7D0FA164B05001E78731E9E413B68D6
:106BF000F6B2191DD878FFF757FB3B682900DA7AFF
:106C0000043303929A79019302920090330020009A
:106C1000059A04F085FD07B0F0BDFFF7B5FF002829
:106C200005D00620FFF7AEFA04000720D8E70820B9
:106C3000FFF7A8FA04000920D2E7C0467464FF1FDA
:106C40007064FF1F70B50A4E040033780D00FF2BEF
:106C50000DD0042004F05CFD011E08D0D023037089
:106C6000CE3B45708370C470307804F0C1FB70BDBA
:106C70002C43FF1F70B5040006200D0004F048FDF2
:106C8000011E0AD0D0230370CD3B8370054B4470A6
:106C90001B688580187804F0ABFB002C01D0FFF74F
:106CA00067FF70BD7464FF1FF8B5264F06003B6890
:106CB0000D001124002B05D10522234B1B78134214
:106CC00002D112242000F8BD204A10241268002AA4
:106CD000F8D01278002AF5D0DB0719D52B789A1E48
:106CE000012A1AD80C2004F0DBFC13243860002899
:106CF000E8D000230A22437029000670023004F015
:106D000097FAFFF75BFF041E0AD0FFF731FFD9E7C0
:106D100000F012FB0028E1D1E4E7002BE2D0D0E73D
:106D20000B4B1B78032BCDD11D20FFF72BFA094B02
:106D300018800028C6D0084B04211878074A04F0B0
:106D40009FFBBFE77464FF1F7164FF1F9064FF1F08
:106D50007064FF1F6E64FF1F9C64FF1F60EA0000E9
:106D6000F7B50193194B14001A78052306000F009C
:106D700012201A4221D0012920D1154B1D68002D67
:106D80001BD002201F2C18D8002C02D0019B002BF6
:106D900013D0104B1F221E706E1C0021300004F017
:106DA0005FFA01992200300004F042FA310020001D
:106DB0002C70002F06D004F0CBFAFEBD064B12203B
:106DC0001D68DCE704F084FBF7E7C0467164FF1F31
:106DD0009064FF1F2C43FF1F8C64FF1FF8B50F4EFC
:106DE00012243368002B17D01B780F3C834213D139
:106DF00000250B4F0221387804F012FD094B0421C5
:106E000038781D8004F00CFD074B28001D80336886
:106E10005C7004F0C5FA04002000F8BD7464FF1F24
:106E20009C64FF1F8864FF1F6E64FF1F70B50128FC
:106E300023D11B4C2388002B03D01A4A1578002D30
:106E400007D0194B1B68002B02D01878FFF7C6FF3C
:106E500070BD3B2B02D93C3B2380F9E7134E022146
:106E6000307804F0DDFCFA222388920002215A4394
:106E7000307804F0E5F92580EAE70B4B1B68002B1E
:106E8000E6D00B4B1B785B07E2D5084B0221187844
:106E900004F0C6FC0022024B1A80FFF769FED7E718
:106EA0008864FF1F6C64FF1F7464FF1F9C64FF1FD6
:106EB0007164FF1FF8B51E4D2868002803D004F048
:106EC0001FFC00232B601B4E3068002803D004F009
:106ED00017FC00233360184F05243B78180020402E
:106EE000234221D0154800F02BFA3B78234213D0DF
:106EF000202004F0D5FB2860002813D02022002198
:106F000004F0AEF9202004F0CBFB041E306005D065
:106F10002022002104F0A4F9002004E0286804F0F5
:106F2000EFFB2C601320F8BD00F00AFAF4E7C0462E
:106F30009064FF1F8C64FF1F7164FF1F2043FF1FBD
:106F400010B50A4C23681A1E0ED0002808D1013053
:106F5000587004F025FA002805D02368002B02D0D1
:106F60000021FFF787FE0122100010BD7464FF1F8F
:106F7000F7B5274E050033680191181E21D05C78C3
:106F8000244F012C30D1FFF7FFFD002825D0200031
:106F9000FFF7F8F80400412814D91F4B0221187894
:106FA0001E4A04F06DFA1E4B3C3C1C8002223368E2
:106FB0005A703B78002B14D128000199FFF75AFE34
:106FC0000120FEBDFA2292004243002AEED0124B6D
:106FD0000221187804F034F9E8E7FFF7D3F802004B
:106FE000F3E700233B70EBE73B78002BE8D103206D
:106FF00004F08EFB011E08D0D0230370CC3B4570FB
:1070000083703368187804F0F3F9FFF7B1FDD7E720
:107010007464FF1F6C64FF1F9C64FF1F60EA000024
:107020008864FF1F10B51749838802008B4220D067
:1070300011D815498B4217D0144900205B1899B21A
:10704000012907D8926811785A425341D8B2FFF704
:10705000F9FD012010BD0E4A00209B1807229BB2AB
:107060009A424041C0B2F5E783681878FFF768FF9D
:10707000F0E7836899785A78090218781143FFF786
:1070800077FFE7E70A20000006200000F8DFFFFF97
:10709000AFDFFFFF014B18707047C0462D43FF1F45
:1070A00010B5064C207001F041FA207804F0B0F9D8
:1070B0000521207800F062FD10BDC0469C64FF1FD2
:1070C0000BB273B50D00002B00DBC4E0884B1878C1
:1070D00004F0D6FA041E0ED00378912B0FD0A22B09
:1070E00000D1A1E0834B1878FF2852D0210004F092
:1070F0007FF900284DD180200002684076BD43789A
:107100000F2B76D013D8052B70D00E2BEAD18088A8
:10711000794B98422BD8794B98421BD8784B9842A0
:10712000E0D1A3681878591CFFF774F838E03E2BBB
:10713000D8D18378032B74D06CD8012B6ED0022B5E
:10714000D0D1704B1B68002B23D05B68002B20D064
:1071500098471EE06C4BC0180C28C3D804F068FB9D
:107160001DC2C2150BC20B0B0B3223C23C00674B76
:10717000C0180728B6D8664B1B68002B09D01B68BF
:10718000002B06D0200098470AE0A3681878FFF784
:10719000C7F8200004F0D4FAADE7A068FFF762F862
:1071A00000289FD0F5E7A3681B78002BF1D0554B42
:1071B0001B68002BEDD01B68002BEAD0210055483E
:1071C0009847EDE74F4B1B68002BE2D01B68002B64
:1071D000DFD021005048F3E7504B1B68002BD8D07C
:1071E0005B68002BD5D021004348E9E7FFF7EAF9B7
:1071F000CFE780884A4B984203D04A4B984200D050
:1072000070E7464B1B68002BC3D05B68002BC0D0D7
:107210002100D5E7153B012BBBD963E7FFF798FAAF
:10722000B7E7FFF77DFAB4E73F4B1B78042B07D194
:1072300000236A4613800179408800F0C5FCA8E766
:10724000364B1B68002BA4D05B68002BA1D001003B
:10725000364898479DE7012421420AD0294B1B68F4
:10726000002B04D05B68002B01D000209847012040
:1072700043E78B070AD5264B1B68002B04D05B68BD
:10728000002B01D020009847022036E70421280077
:1072900008400D4200D131E7254E3388002B21D024
:1072A000013B9BB23380002B1AD1FFF7DBF800289B
:1072B0000AD0204B1C70164B1B68002B04D05B6857
:1072C000002B01D020009847FFF7C6F8694601F06F
:1072D00001FD6846FEF7FEFF1D20FEF753FF3080DC
:1072E00004200AE7024B187804F09AFAF8E7C0463F
:1072F0009C64FF1F2D43FF1F0E2000000120000093
:10730000091000009464FF1FFEDFFFFFAFDFFFFFE7
:107310009864FF1F0C2000000B2000007C64FF1FFE
:107320000D200000132000007164FF1FFFFF00000C
:107330006E64FF1F6C64FF1F10B501F09BF910BD58
:10734000014B18607047C0469864FF1F0B880020EF
:10735000162B01D817230420014A13807047C0461A
:107360004664FF1F00207047074A030011888142CE
:1073700007D091880020994202D101308000101876
:1073800070470020FAE7C046A464FF1FF0B58F786D
:1073900006000D00C5B01E2F15D1FFF7E5FF051E35
:1073A00003D10024200045B0F0BD00223B00310095
:1073B000C078009200F0B2FB0400A81C00F0D2FBE1
:1073C000FF23EB70EEE7264B062403931B78FF2B7D
:1073D000E8D0182FE6D87B08224A013BDB00029256
:1073E0009A589446002ADDD0029AD3185B68002B85
:1073F000D8D00878002802D14B78012B02D106247E
:10740000122FCFD107AFAB88697800976446AA687E
:10741000A047041EC6D1AB78029A5B08013BDB0093
:10742000D318390030005B689847041E0BD1AB7845
:10743000042BB6D0039A310010782200009700F098
:107440006DFB0400AEE76A78002AABD1AA7805A9E3
:107450003B88087130000A704B80FEF747FBA0E7BD
:107460003043FF1FFCB900111D4B37B50500984292
:107470000BD000290AD1FFF777FF002805D1194862
:10748000FFF772FF002800D0058037BD01291AD10F
:10749000FFF76AFF041EF8D001235B420380A37844
:1074A000FF2BF2D0FE2B07D00023E07814220093AC
:1074B00029001E3300F032FBA01C00F053FB012317
:1074C0005B426380E1E70229DFD1013901F0BEF8B8
:1074D0000028DAD12800FFF747FF041EDFD1D4E7E8
:1074E000FEFF0000FFFF0000022210B5074B5242D2
:1074F0001A80074801325A809A80DA8000F07EFABA
:10750000044801F025F8002010BDC046A464FF1F08
:107510008D730011697400110388F7B50400002B06
:1075200002D102252800FEBD4268022113782548B9
:107530005268FEF7A5FD00282ED0234F01253A887A
:10754000002AEFD0802321885B0201259B1A9942F3
:10755000E8DC0C2004F0A4F8061E31D03B88228819
:107560009C4600231800019561469DB2491989B2D5
:10757000AA421BD8002801D062443A800023300080
:10758000082208C0210003F053FE104A1368002BA4
:1075900013D100251660C5E76268022113780C48F4
:1075A0005268FEF76DFD0028C7D1BAE760681D017B
:1075B0004019418101330198D6E71A001B68E6E7BC
:1075C0001325AFE76ABA00112E43FF1FA064FF1F07
:1075D00068BA0011014B18707047C0463043FF1F56
:1075E00014230A0010B51A40194204D001221021B8
:1075F00001F048F810BD4B06F9D401208843400043
:10760000F8E710B514008B0604D50122102101F013
:1076100039F810BD08230A001A40194202D14BB2B2
:10762000002B0FDA102101F02DF8002808D02300DC
:10763000F2331B78002BECD0F1342378012BE8D106
:107640000020E6E703208907FAD4E2E7F0B51F003F
:10765000184B85B01C68019002910392002C27D131
:10766000200005B0F0BDA5683301ED186B89019AC3
:10767000934211D3029A93420ED8002F04D10A9B51
:10768000002B10D12C00EBE73B002978039A6868A7
:10769000FEF7F6FC0028F2D10136B6B2A388B34259
:1076A000E1D82468DAE7A3680A9A5B891380E9E7DE
:1076B0000026F3E7A064FF1F37B50C000A8849884D
:1076C0000123914217D3002A15D0651D23792A0082
:1076D00002210A48FEF7D4FC102300280BD023799E
:1076E0006188208800242A000094FFF7AFFF0A2356
:1076F000A04200D0230018003EBDC0466ABA001167
:1077000013B50A0008884988012388420BD800284D
:1077100009D00024137905320094FFF797FF0A235C
:10772000A04200D02300180016BD13B50A00088837
:107730004988012388420BD8002809D000241379F6
:1077400005320094FFF782FF0A23A04200D02300F5
:10775000180016BDF0B58BB003904A8808880E005B
:107760000123824255D3002853D00023012704ACC3
:1077700023700022718813000092FFF767FF051E37
:107780003ED02078002835D12B78022B18D1677095
:107790006A8983000130E31880005A8069680222F8
:1077A000201803F045FD23780133DBB22370042B4E
:1077B00019D93B006889013080B2002BD9D01FE075
:1077C00002236370122358436A89231804305A80B5
:1077D00069681022201803F02BFD23780133DBB2F7
:1077E0002370002BE5D10C4A6B899B185A425341F8
:1077F000DBB2DFE76378012BE4D12B78022BC7D013
:1078000022780A23002A04D021000398FEF798F971
:10781000002318000BB0F0BD0100FFFF0F4BF0B5C7
:1078200004001868002816D083685D89A54207D82F
:107830008288AE18B44203DA12019A18934201D139
:107840000068EFE71E005F891036A74204D10029C7
:1078500000D00D801800F0BD3300EFE7A064FF1FDB
:1078600070B505000C0008880021FFF7D7FF030062
:107870000120002B04D022002800197AFFF7C1FE56
:1078800070BDF7B50C00002501902300EE331B7886
:10789000AB4201D800200AE06B00E65A002130001C
:1078A000E718FFF7BBFF002802D126800130FEBD9C
:1078B000017A0198FFF794FE002802D03B882380CC
:1078C000F5E70135EDB2E0E710B5040008880021C6
:1078D000FFF7A4FF03000120002B03D02000197A3A
:1078E000FFF77EFE10BD0000054B1B68002B01D189
:1078F000180004E09A6852898242F6D1988870474D
:10790000A064FF1FF0B50E27002687B0039302ABDB
:10791000FF183E8005001F4B40891400984207D095
:107920002B78013000976A6880B2FFF78FFE06005F
:1079300002212B7818486A68FEF7A2FB00280FD0B6
:107940006C892000FFF7D0FF002802D0013C041909
:10795000A4B2039B002B00D01C80300007B0F0BD08
:1079600002212B780D486A68FEF78AFB0028E7D1D0
:1079700002212B780A486A68FEF782FB002807D0AC
:10798000002EDED03B88A342DBD17489013CDFE7C7
:107990006C89DEE7FFFF00006ABA001168BA0011C7
:1079A00066BA001110B50C00FFF7DEFC03000220E0
:1079B000002B0AD0002C00D023609B781720FE2BD0
:1079C00003D00138FF2B00D1002010BD73B50D008E
:1079D00001A904001600FFF7E5FF172805D0002EC7
:1079E00004D129002000FEF727F976BD01221021DD
:1079F000200000F047FE0028F3D0F6E7014B1860A6
:107A00007047C046B064FF1F37B56B469D1D01002F
:107A100004000222280003F0DBFE2B88B02B0ED1DD
:107A20002379122B09D12300FA331B78012B06D1BD
:107A30000121608800F0E0F801E01B2BF8D037BD91
:107A400010B5054B0421187000F098F8FFF74CFDB5
:107A5000FEF770FB10BDC046B464FF1F0020F0B5F8
:107A60000BB20F0087B0834234DA274B187803F04B
:107A700007FE051E2BD00378A02B25D103AE3100C5
:107A8000FEF7E4F8041E0BD1B378DB0724D51F4BB7
:107A900006341B68002B03D0310068889847040027
:107AA000A868002801D003F063FD002C08D1184A13
:107AB000039B1340174A934206D0B3781B2B03D085
:107AC0000121688800F098F8280003F039FE802032
:107AD0000002784007B0F0BD0F4B1B68002B10D0A0
:107AE000310068889847041EDAD07378002BD7D10C
:107AF000B27801A90A704B800C716888FDF7F6FF17
:107B0000CEE70624F1E7C046B464FF1FAC64FF1F54
:107B100000FFFF0000011200B064FF1FF7B50190E5
:107B2000FC200D0017001E0003F0F2FD04001320DE
:107B3000002C12D0B02320002370089BF422677021
:107B4000658026710830002B08D0190003F070FB07
:107B50002100019803F04CFC0020FEBD089903F0C1
:107B60007FFBF5E710B5041E06D00078FD2803D88A
:107B700003F06EFEFF23237010BD00000A1F93B2B6
:107B800010B504000220032B05D882400020024BD0
:107B9000D1529B189C7010BDD464FF1F0B8870B528
:107BA000043B04000D000220032B0BD80121200010
:107BB00000F04CFD03001420002B03D0290020000E
:107BC00000F0DEFB70BD000007B51300034A009211
:107BD0000A00012100F02CFC0EBDC046057E0011FC
:107BE00007B5019203220092024B0A00122100F015
:107BF00049FC0EBD837E001107B56B4601AA1180BA
:107C00000449D88008780633012802D1190003F00E
:107C10002FFC07BDB564FF1F0C4B10B51870002377
:107C2000FF210B4A1380138193819380094A53806B
:107C30001370517293819372D174D38213755177FB
:107C400003F0C6FB00F0FCF910BDC046E464FF1F62
:107C5000D464FF1FB664FF1FF0B58DB06B460020E3
:107C600003910C229B5E834200DBB0E05D4B1878F1
:107C700003F006FD051E00D1A4E00378902B00D090
:107C80009DE006AF01004688380000F013FA7968DD
:107C90000400002900D19CE03B88052B6ED13B8974
:107CA000032B1CD905AC200000F0A2F86288172A2B
:107CB00061D83989131D994231D17968237804310B
:107CC0000291D90738D5607800F08EF9071E06D0EA
:107CD000002303712378012B08D0132B23D0A8682D
:107CE000002800D178E003F043FC75E06288029937
:107CF00009A800F0A6F80290380000F08BF909AA54
:107D00002378387A0192002231000092029A00F022
:107D100012F9380000F064F9029B002BDFD030002C
:107D200000F080F9DBE70378032BD8D16288029951
:107D300009A800F0D6F8DEE7122B13D1029909A8A2
:107D400000F0B5F8021EEAD127498B88002BC6D077
:107D5000887909A92378019161780091310000F0B8
:107D6000EAF8BCE7002302AA93833000617809AAED
:107D7000FFF72AFFB3E71D4B0993F6E7042B02D068
:107D80009A1F012AABD8184A043B9B00995A002934
:107D9000A5D0D218907831003A0000F0AEF8002853
:107DA0009DD13B88042B03D001213000FFF724FF35
:107DB000012C04D1A868002801D003F0D9FB2800C9
:107DC00003F0BEFC8020039B0002434018000DB06E
:107DD000F0BD012800D182E701213000FFF70CFF40
:107DE000EDE7C046E464FF1FD464FF1F01001700E5
:107DF0000B7803704B784370CB788A781B0213435F
:107E0000438070470A88030002700A88120A427091
:107E10000A88012A06D14A8882704A88120AC270EA
:107E20000420704702208242FBD14A8804309A70B5
:107E30004A88120ADA708A881A718A88120A5A7174
:107E4000EFE710B50400012082420CD94B780A7884
:107E50001B0213432380834206D1CB788A781B020E
:107E600013436380002010BD022BFBD1CB788A78AE
:107E70001B02134363804B790A791B021343A380CF
:107E8000F0E70B8803700B881B0A43704B888370E4
:107E90004B881B0AC3708B8803718B881B0A437144
:107EA000CB888371CB881B0AC371082070470300FD
:107EB0000120082A14D14A780878120202431A8055
:107EC000CA788878120202435A804A7908791202E5
:107ED00002439A80CA798879120202430020DA802C
:107EE000704710B504000120022A05D100204B780C
:107EF0000A781B021343238010BDF8B5060010203A
:107F00000F00150003F004FC04000120002C0ED02B
:107F1000A0230C22290023806780201D002D07D07C
:107F200003F086F92100300003F062FA0020F8BD6A
:107F300003F096F9F6E7F7B51E00009008AB1420A1
:107F400017001D78019103F0E3FB041E12D0A22359
:107F50000370019B47704380099B057146710C2299
:107F60000830002B07D0190003F062F921000098B7
:107F700003F03EFAF7BD099903F072F9F6E737B559
:107F8000041E0FD04388002B0CD00025C18813237A
:107F9000007A172201950095FFF7CDFFFF2365803A
:107FA0006372257037BD000010B50C4904004A8883
:107FB000002A09D08B89002B05D00020CB8A022211
:107FC000834201D010BD012213000A204343002048
:107FD0004032C854C81842800472F3E7B664FF1FE9
:107FE0000023438003707047094B00211A0010B52D
:107FF0005C88002C06D01C79844203D10A234B43B1
:10800000D01810BD01310A330329F1D10020F8E75F
:10801000B664FF1F10B50400407A03F019FCFF237B
:10802000637210BD7047043010B580B203F008FAD7
:10803000002803D00421494203F05AFB10BD000080
:1080400070B50025104CA0682580A581A580A842A8
:1080500002D003F08DFAA56000250C4C0C4B606D2E
:108060001D80230058331D70A84202D003F080FA0F
:10807000656500256068002801D003F079FA0135B4
:1080800008340A2DF6D170BD7C65FF1F2065FF1FE7
:108090007065FF1F70B5041E09D1054D2880A881A9
:1080A000A880A868002802D003F062FAAC6070BD16
:1080B0007C65FF1FF0B54B8885B0019300234360BA
:1080C0000A7905000F00022A00D07BE0CA88032A43
:1080D00017D98B685E7819783602DC78D8790E4328
:1080E00099781B7A24021B020C43034353495BBA61
:1080F0000B80331D93421ED1042C04D0631F022B2E
:108100000ED9012015E0019A4D4B1201D35A002BD4
:1081100006D00198FFF7BEFF4A4A13690133136185
:108120000421B8682E812C80494203F0E1FA68608E
:10813000002005B0F0BD434D042C06D0631F022B78
:108140000FD9EB680133EB60DBE7019A3C4B12017E
:10815000D35A002B05D00198FFF79CFF2B69013300
:108160002B61374B30000293019B029A1B01019354
:10817000002301998C468B52130063449C80039327
:108180009E81FFF750FF039B041E986016D00421C8
:10819000B868494203F0ACFAFA880100043A2000BA
:1081A00003F046F80199029AFB888A5A043B9B180F
:1081B000029A8B522B6801332B60A2E7AB69013323
:1081C000AB619EE71E4B0293019B1E01029BF35A7B
:1081D000002B2DD002998C19A068002828D0012AE4
:1081E00026D1FA889B189BB27352A189994217D362
:1081F0009B1AC018B96803F01BF8029BA289F35AB6
:10820000934200D07DE700222B81A3882B80A368B6
:108210006B60029BF2520B4A53680133536070E764
:10822000084A9368013393600198FFF733FF68E7CA
:10823000044A536901335361F6E7C046E664FF1F01
:108240007C65FF1FEC64FF1F70B5051E15D10B4C3C
:108250000B4B1880230058331870606D002802D033
:1082600003F086F96565250050356068002801D067
:1082700003F07EF90834AC42F7D170BD2065FF1FD2
:108280007065FF1FF0B51700A12285B09200019321
:108290004243394B06001B680C009B18D933FF334F
:1082A0001D78FDF741FF0430854204DD3000FDF705
:1082B0003BFF0430C5B2BD4207D33A000021300075
:1082C000019B03F08DFA05B0F0BD2900380003F0E2
:1082D0007FF92300C6B250331E700393019B29001F
:1082E0006365380003F064FACBB20293002B02D02E
:1082F000039B01361E7000262300503303931B7826
:10830000B34204D8606D002831D10020DBE7029A27
:108310002800002A04D0013B1000B34200D02800FE
:10832000F700E719387002F0C3FF786000280ED01C
:108330003A78019902F07CFF019A3B780136D31814
:108340000E4A0193D369F6B20133D361D4E7039B9C
:1083500018706065A74205D1084A1320D36A01331B
:10836000D362B0E7606803F003F90834F2E703F082
:10837000FFF800236365C8E73409FF1FEC64FF1FA3
:10838000F7B50D0007000421686803F0B1F92B89E7
:10839000040003702B891B0A43702B8883702B8881
:1083A0001B0AC3702E8902250436F6B2F42E15D8A6
:1083B0001B4B9F4214D10C2003F0AAF91135011E6A
:1083C0000CD0902303708E3B0371043B4380154B0C
:1083D0008460C680187803F00BF800252800FEBDE5
:1083E0005C237B43104AD3180093583301931B78C6
:1083F000002B0FD10300320038000099FFF742FF35
:10840000019B05001B78002BE8D13800009903F090
:1084100007F8E3E7054A0725536A01335362DDE7AE
:10842000FEFF0000E464FF1F2065FF1FEC64FF1FD8
:10843000F0B587B0009017200F0016000193FFF7EA
:10844000F2FD1325041E19D00C98031E02D00199C9
:10845000201D9847030AE370052302AAA070043088
:10846000908127700098667003A993800494FFF7A9
:1084700087FF051E02D0200003F07AF8280007B01D
:10848000F0BD0000F0B587B01F000CAB1B78039166
:10849000059301210DAB06001C78049200F0D6F87C
:1084A0001425002821D02000FFF77EFD0135041E91
:1084B0001BD01149059B0A7803700132D2B2131EFA
:1084C000C68001D101231A000B7022713000049B79
:1084D00003990097FFF7ACFF051E09D12300210087
:1084E0000648074A093302F0B3FF280007B0F0BD81
:1084F000002363802370F8E7E864FF1F7F7F00118B
:1085000030750000F8B505000E00064C064F2368D4
:10851000002B02D03100280098470434BC42F6D129
:10852000F8BDC0468C65FF1FA065FF1F0123064AEA
:108530005B425380002313715362044A13605360FB
:108540009360D36013617047A065FF1F8C65FF1FA8
:108550000200002310B506499C000859002801D1EB
:10856000625010BD0133052BF6D11320F9E7C04648
:108570008C65FF1F034A5388181A434258414042F2
:1085800010407047A065FF1FF0B585B002930AAB9D
:108590001F780CAB1B88009008000E00019203931B
:1085A000FFF7E8FF05001120002D1BD10E48FFF753
:1085B000E1FF04001520002C14D006220B99A771AE
:1085C000E01D02F035FE019B30002371029B290063
:1085D0006371009B66802370039B6562E381FFF7F4
:1085E00091FF280005B0F0BDFFFF000010B5FFF7B8
:1085F000C1FF04000220002C12D060880121FFF787
:1086000081FF606A002801D003F07AF82822002157
:10861000200002F025FE012300205B4263802071D0
:1086200010BD000030B5074A074C5588010013788B
:108630000020A54204D05B1A59424B4158421040D9
:1086400030BDC046A065FF1FFFFF0000084A10B5FF
:1086500001230C00904208D0FFF78CFF031E04D0CA
:10866000037923405A1E9341DBB2180010BDC04667
:10867000FEFF0000024B1879431E9841C0B27047BC
:10868000A065FF1F70B504000D001600FFF772FF14
:10869000002804D10D4B9C4200D0143070BD416ABB
:1086A00003790520002907D012221A40102A02D18E
:1086B0000520002EF2D10F20DB06EFD5897E0C209D
:1086C000A9428941494249420840E7E7FEFF0000CC
:1086D000030010B5002800D110BD0348034A4188AB
:1086E0009142F9D09847F7E7A065FF1FFFFF000010
:1086F000002330B5C45CCD5C6C40D4540133102BE6
:10870000F8D130BD0F23002210B5C45C64002243B1
:10871000CA54C25CD209013BF7D210BD020001006D
:1087200010B52032103102F0F3FE10BDF0B58BB061
:108730000390102005931700049102F0B1FF009000
:10874000102002F0ADFF009B13240190002B05D0F8
:1087500000280CD11324009802F0D2FF019B002BBB
:1087600002D0180002F0CCFF20000BB0F0BD1020AA
:1087700002F096FF0600102002F092FF132405007D
:10878000002E00D1AEE0002819D01022002102F006
:1087900067FD32002900039802F0BAFE041E0ED1D4
:1087A00033787F2B51D830000099FFF7ABFF009B47
:1087B0001B787F2B53D801990098FFF7A3FF300057
:1087C00002F09EFF002D02D0280002F099FF002C3D
:1087D000C1D1102002F064FF0600102002F060FFFB
:1087E0000290002E7CD0002878D03A000F3223006F
:1087F0000125121105D00F333B4015B25A425341A7
:108800001BB26A1E1201002B33D0049BD2B29818FF
:108810000099029AFFF76CFF013D10220021300001
:1088200002F01EFDADB2049F2D017D19AF4242D072
:10883000002C33D0300002F063FF029B002B00D1EC
:1088400089E7180002F05CFF85E729003000FFF798
:1088500059FF28002549009AFFF74AFFA7E729009A
:108860000098FFF74FFF28002049019AFFF740FFCB
:10887000A5E70F210F4004998A18D9B28F4208D971
:10888000D15C06A819540133102BF6D1029A019934
:10889000C0E7791A48424141C901F2E73900300086
:1088A00006AAFFF725FF3200039806A902F030FE62
:1088B00010370400BAE7002CBCD13000029906AA98
:1088C000FFF716FF320006A9039802F021FE0822E6
:1088D00004003100059802F0ABFCABE71324A9E7D4
:1088E0001324AAE7002800D06EE733E770BA00111E
:1088F000F0B58BB00F0016000225009000283FD085
:10890000002A3DD00B1DDBB21800029302F0C8FE16
:108910001135041E34D0FDF747FD05003A000099DB
:10892000201D02F04DFFEBB20393E3702B0CDBB282
:108930002F0A00936370FFB22B0E2370A770019370
:10894000FDF72CFD1022010006A802F039FF2100DE
:10895000029A04AB06A8FFF7E9FE051E0DD1039BA2
:1089600008223370009B04A9B370019B7770F370E9
:10897000301D02F025FFFDF71DFD200002F0C0FEB6
:1089800028000BB0F0BDF0B58FB00D00149E039021
:1089900004920593002A03D1022420000FB0F0BDF9
:1089A000002EF9D00398FFF7E5FD1424071EF4D03C
:1089B0007278337812021A43B3781B041343F278A7
:1089C00012061A43036A0192934201D30133E3D1A1
:1089D000002D03D03B7901249B07DED5082200211E
:1089E00006A802F03DFC059B13240433DBB21800FB
:1089F000029302F055FE051ECFD0059A049904306B
:108A000002F0DEFE04223100280002F0D9FE390017
:108A1000102210310AA802F0D3FE2900029A06ABF8
:108A20000AA8FFF783FE041E0FD1082206A908A892
:108A300002F0C6FE0822311D08A802F059FD0128E7
:108A400007D101990398FDF7C9FC280002F058FEF0
:108A5000A3E70124F9E7000070B51C4C050023686A
:108A6000181E10D0002D14D11A78002A0CD1981C91
:108A7000083202F0DDFB02F0EBFD0135002808D1E1
:108A800023681D70012070BD0A331800082202F00F
:108A9000CFFB2368002BF5D0122002F039FE061E12
:108AA0000DD0C123216803704570023110220230BD
:108AB00002F0BEFB23683100587802F099FC206870
:108AC00002F01EFE00232360DCE7C046C865FF1FDE
:108AD000F8B504002020FDF755FB0D4EA700BB594B
:108AE0000500002B0DD000280BD0D878FF2809D125
:108AF00008492A000C55F35907480333611802F05E
:108B0000A7FCF8BD290002F00BFD0028F0D1F8E722
:108B1000E465FF1FCC65FF1F299D001170B5064D50
:108B200084006359002B05D0D87802F091FEFF2213
:108B30006359DA7070BDC046E465FF1F70B506006A
:108B40008CB00C00150000213022684602F088FB32
:108B500031001022684602F033FE1D20210003225E
:108B6000684402F02DFE6846FFF7D8FD2D21040071
:108B700003222800694402F023FE20000CB070BDDF
:108B8000F0B50700160097B001931CAB1D7830229A
:108B90001EAB00910AA800211C7802F061FB102294
:108BA00039000AA802F00CFE1022002102A802F0EF
:108BB00057FB0722310002A802F002FE072202AB97
:108BC0009818631E9C41019902F0FAFD02AB9C7358
:108BD0002B005A1E934102AAD3730021102206A82B
:108BE00002F03EFB06221D9907A802F0E9FD1A20BB
:108BF00002ABC01806221F9902F0E2FD1022009974
:108C00000EA802F0DDFD102202AB0EA908781C7838
:108C1000013A6040D2B2087001330131002AF5D127
:108C20000AA8FFF77BFD102212A904000EA802F08B
:108C3000FFFA102206AB0EA908781D78013A6840A9
:108C4000D2B2087001330131002AF5D10AA8FFF72A
:108C500065FD044310222098E4B212A902F0B0FD91
:108C6000200017B0F0BD70B50E0014008CB00100EC
:108C7000102268461D0002F0A3FD3100082204A85E
:108C800002F09EFD2100082206A802F099FD684628
:108C9000FFF744FD04001022280008A902F090FD0F
:108CA00020000CB070BDF8B506000D000024371987
:108CB000AC4200D3F8BD02F043FC030A3B70631CD6
:108CC000DBB201379D4203D90234F054E4B2EEE73F
:108CD0001C00EDE773B506000C000225002819D032
:108CE000002917D0032101A8FFF7DDFF6B469A7911
:108CF0003F231A40013313436A463000937101A9A0
:108D00002200FFF71BFF051E04D10322E01C01A96E
:108D100002F08EFA280076BD03785807DA08C00FF3
:108D2000D20080009B0710439B0F1843C0B27047CE
:108D300007230B40C908C9000B43037070470000AC
:108D400070B50400FFF7EAFE134DA4006359002B31
:108D500021D0186A002801D002F0D2FC2B59986E5D
:108D6000002801D002F0CCFC2B59D86E002801D08D
:108D700002F0C6FC2B59186F002801D002F0C0FC8D
:108D80002B59586F002801D002F0BAFC285902F084
:108D9000B7FC00232B5170BDE465FF1F0E4B800014
:108DA000C35870B50C00002B0FD09D68002D0CD05F
:108DB0002B78201D0B706B784B70A97CFFF7B8FFE8
:108DC0002B7E23726B69E36070BD102200212000AE
:108DD00002F046FAF8E7C046E465FF1F014B186051
:108DE0007047C046E065FF1F074A030080008258B5
:108DF00010B5002A06D0D088984203D1012901D1AC
:108E0000FFF79EFF10BDC046E465FF1FF0B5264E7C
:108E100095B087000B93BB590500099112200A9267
:108E2000002B31D0D888FFF7A5FB04001420002CBC
:108E30002AD0280010A9FFF7B1FFBB591E781D6A80
:108E4000002E23D00895FDF7EFFA07000020FDF76C
:108E5000F1FA0790A379E61D069310AD0CA90898C6
:108E600000F0E2FA0EA9280000F0D7FA0B9B0A994D
:108E70000493069B09980293079B0396019300971E
:108E80000EAB0CAAFFF77CFE15B0F0BDFDF7CCFAD7
:108E900006903000FDF7CEFAE31DA779079310ABDB
:108EA00006000893DAE7C046E465FF1F30B50C4CB6
:108EB00085002A59030085B00120002A0ED0180031
:108EC0006946FFF76BFF2B591A78D888054B002AA3
:108ED00000D1054B6A46072100F0D9FB05B030BD33
:108EE000E465FF1F1B9400112994001130B5094C53
:108EF0008500295985B010226846253102F098F97D
:108F00002A591121044BD0886A4600F0C0FB05B0F5
:108F100030BDC046E465FF1FC594001130B5094C53
:108F20008500295985B010226846353102F080F954
:108F30002A591121044BD0886A4600F0A8FB05B0DD
:108F400030BDC046E465FF1F03950011F7B54D4FD6
:108F500086001020F4590D0002F0A2FBF3592062A4
:108F6000186A132200286CD0033A29009C6802F08A
:108F70005FF9F3591A780192002A58D11E6A227DAE
:108F8000317B944651400122019F114201D1674635
:108F90001740217D914339432175377B4F40BC46B3
:108FA00060460027800701D44F08174001210220A6
:108FB0008F40227D82433A432275377B5740BC461F
:108FC00060460027400701D497080F400420227D07
:108FD000BF0082433A432275627D00279446604673
:108FE000727B42400A4201D167460F400121627DF7
:108FF0008A433A436275777B5740BC4660460027F8
:10900000800701D457080F400220627D7F00824311
:1090100017436775767B00227E40760701D4BA0835
:109020000A400426617D9200B1430A4362756A7862
:10903000002A08D06278002A05D005220533DA77A5
:1090400000221000FEBD04222979114205D1A17C25
:10905000114202D10533033AF1E7019A21782C78C5
:10906000002A02D10A002100140018220429E8D89D
:10907000042CE6D805206043034A05331218525CDD
:10908000DDE7C046E465FF1F80BA001110B50A0095
:109090001121024B00F0FBFA10BDC0465F95001194
:1090A0000B0030B587B001AD2B806B46040011007A
:1090B000981D082202F0BCF82A000B212000024B68
:1090C00000F0E5FA07B030BD8795001110B50A0031
:1090D0001121024B00F0DBFA10BDC046DB950011F8
:1090E00013B50B0011006A4613706B46040006228C
:1090F000581C02F09DF86A4608212000014B00F040
:10910000C6FA13BDFB95001110B50A001121024BE0
:1091100000F0BDFA10BDC0464B9600117FB50500AA
:109120000B4BAA00D4580800002C0FD0666F237F89
:10913000E28821780396266F0296E66E0196A46E69
:109140000094FDF709FC2800FFF7FAFD7FBDC0463B
:10915000E465FF1F10B51721FFF7E0FF10BD000009
:1091600070B50A000D00064B0221040000F08FFAD2
:10917000060029782000FFF7D1FF300070BDC046FF
:109180002B95001170B586B000236A461370836872
:1091900004001D78681E0A2859D801A902F0A0F918
:1091A000060633373B3F43474B4F5300180000F050
:1091B00042F9062312284BD000281BD16088FFF704
:1091C000D9F90823002813D04279002A47D1264B29
:1091D0001A78072312070BD5244B1A680723002A95
:1091E00006D01668002E03D0290001AAB04703005C
:1091F0006A4613706B461B786088002B2AD1FFF7F4
:1092000067FC06B070BD180000F06CF9D4E71800D8
:1092100000F087F9D0E7180000F093F9CCE71800C8
:1092200000F0ADF9C8E7180000F0C3F9C4E7180072
:1092300000F0F6F9C0E7180000F0F6F9BCE71800F6
:1092400000F013FAB8E7180000F013FAB4E70723A8
:109250006A46137069466088FFF782FFD1E70523ED
:10926000012AC5D1024BB8E77164FF1FDC65FF1FFF
:10927000E065FF1FF8B52C4F8600F35904000D0080
:10928000002B40D0DA8882423DD15A78062A33D169
:109290001A78002A2ED0012099681A6A097D0142A5
:1092A00006D0157B054203D007225A700120F8BD75
:1092B0000220014204D0157B054201D00922F4E7C7
:1092C0000420014204D0127B024201D00B22ECE7C1
:1092D000164B1B68002BE9D05B68002BE6D0200002
:1092E0009847BB5900215B78122BDFD12000FFF794
:1092F00015FFDBE70E4BECE7112A04D1002900D063
:1093000032252900F2E7002D08D12000FFF732F9BD
:10931000002803D010230279134303712100280091
:10932000FDF798FAC2E7C046E465FF1FDC65FF1F42
:10933000E065FF1F70B50E4E8500AB590400002B91
:1093400013D01B78002B11D10A4B1B68002B04D0C3
:109350005B68002B01D02000984773595B78122B73
:1093600003D100212000FFF7D9FE70BD024BECE7CE
:10937000E465FF1FE065FF1FDC65FF1F094B8000F0
:10938000C3581020002B0CD01A6A002A09D09B6801
:10939000002B06D0127A1B7E101C9A4200D9181C92
:1093A000C0B27047E465FF1F70B503000D001400E4
:1093B0000220002A30D000292ED013700B78081D0F
:1093C00053704B789370FFF7A7FCE07001200221E7
:1093D0002B7A23716B7B034063716A7B0A401343D2
:1093E000042263716E7B1640334363716E7BF60813
:1093F000F600334363712B7B0340A371287B01404C
:1094000000200B43A371297B0A401343A3712A7BDD
:10941000D208D2001343A37170BD10B50A00010039
:109420000120FFF7C1FF10BD10B50A0001000220A6
:10943000FFF7BAFF10BD70B506000C000220002E29
:1094400030D000292ED07378201D0B70B3784B706C
:10945000F178FFF76DFC01223579257271794B1097
:1094600008001340934010400343881010408000D0
:10947000C9080343C9000B436373B1794B1008005B
:109480001340934010400343881002409200C908E3
:109490001343C9000B4321202373FCF773FE85425D
:1094A00001D2122070BD2220257AFCF76BFE854286
:1094B000F7D823781820042BF4D86378012BF1D83F
:1094C0000020EFE7030010B50220002909D0002B8F
:1094D00007D00322481C0A7019000D3201F0A8FEC3
:1094E000002010BD03000222080010B5002B06D09A
:1094F000002904D00E32591C01F09AFE00221000FF
:1095000010BD030010B50220002909D0002B07D0A0
:109510000422481C0A7019000C3201F089FE002058
:1095200010BD10B5FFF7DEFF10BD030002200029BB
:1095300006D0002B04D0052200200A701B784B7047
:10954000704703000220002B08D0002906D05B786A
:1095500000200B70013B082B00D918307047030026
:1095600010B50220002909D0002B07D00622481C84
:109570000A7019000A3201F05BFE002010BD10B520
:10958000FFF7B0FF10BD02000B00022010B500294C
:109590000ED0002A0CD0072119701188597011883B
:1095A000090A997011180822D81C01F041FE002008
:1095B00010BD03000A00022010B5002B0CD00029BA
:1095C0000AD099785878090201431180901CD91C5F
:1095D000082201F02DFE002010BD030010B502206E
:1095E000002909D0002B07D00822481C0A70190056
:1095F000921801F01DFE002010BD02000B00022099
:1096000010B500290BD0002A09D009211970117852
:1096100018185970511C062201F00AFE002010BDD6
:1096200010B5FFF75FFF10BD02000B00022010B560
:10963000002A09D0002907D0517819701118062284
:10964000581C01F0F5FD002010BD030010B50220EC
:10965000002909D0002B07D00A22481C0A701900E3
:10966000063201F0E5FD002010BD10B5FFF73AFF0E
:1096700010BD02000B00022010B5002A06D0002900
:1096800004D018005178FFF753FB002010BDF0B54F
:1096900085B017001E006A46062305000800918168
:1096A0009380FEF7C0FC1324011E02900CD03800FA
:1096B000B047041E05D1280001A9FEF76FFA041E69
:1096C00002D0029801F054FF2800FFF701FA2000B1
:1096D00005B0F0BDF0B504008BB00191150000217C
:1096E000102202A801F0BCFD334EA700B859002893
:1096F0003CD0C388A34239D10378002B36D14278BD
:10970000062A18D102000100553235310C3006AB63
:10971000FFF7A9FA002829D12000FFF72FFE020049
:1097200006A902A801F084FD200002A902F038F881
:1097300001200BB0F0BD816E002917D00B8A112AD1
:1097400028D19D420ED101981231093A01F0D0FE84
:10975000012807D1BB5920009D6EFFF70FFE29009D
:109760000200DEE732212000FFF7D8FC2000FEF7E0
:1097700001FF061E1BD0416A002918D00B8AAB429C
:1097800015D108220198123101F0B2FE01280ED144
:10979000716A0AE09D42E9D108220198123101F074
:1097A000A7FE0128E2D1BB59996E8A7EB9E7200055
:1097B00001F07EFEBCE7C046E465FF1FF0B56B4DCF
:1097C00087007E5985B0337802900393002B00D038
:1097D00087E0B368346A01937078062817D10122B4
:1097E0001B7D134202D0217B114218D10222134269
:1097F00002D0217B114251D10422134203D0237B9A
:10980000134200D08BE0019B5A7DEB5991E0073861
:109810000428F8D801F064FE032E42678300B36E7B
:10982000002B03D11C2001F03BFFB066EB599C6E6E
:10983000002C1CD010220021200001F011FD029804
:10984000FFF79CFD01002000FFF72DFA01F078FEE4
:109850002082200008211230FFF725FA0298FFF736
:109860008DFDA076EB592100D888FFF70FFC082268
:10987000EB591CE0B36E002B05D01A00198AF08852
:109880001232FFF70DFC0222019B197DEB591142A8
:109890003DD0207B10423AD0073208E0F488FCF734
:1098A000DBFD01002000FFF711FC0A22EB595A7082
:1098B000029B9C002A595378073B042B11D8D0886F
:1098C000FEF758FE00284ED0C3895A08D2182849FE
:1098D000029B0298CB542B5941180433254801F0C0
:1098E000B7FD05B0F0BDFCF79FFD030001208342EA
:1098F00001D100200393EB59DE88FCF79BFD03990F
:1099000002003000FFF7ECFB019AEB59117D0422B5
:1099100011420CD0217B114209D00B22C7E7F688F7
:10992000FCF73CFD01003000FFF7EEFB6BE7019A0E
:10993000527D01210A4204D0607B084201D00C22F2
:10994000B5E702210A4204D0607B084201D00E2212
:10995000ADE704210A4204D0627B0A4201D0102202
:10996000A5E71222A3E7FA225200B0E7E465FF1F41
:10997000E865FF1F339D001110B5064B1A780423CC
:10998000100018401A4200D00348FFF727FA0020C1
:1099900010BDC0467164FF1F3443FF1F70B5040043
:1099A000FFF7D4FA051E43D12000FFF77FFA234EBC
:1099B000A400A0598268937CDB0708D50321036AC1
:1099C0001B790B40012B02D1017F0B430377431D11
:1099D000D97F8B1E022B0DD8022900D00121C0880F
:1099E000FCF790FF042133591A7F59700A431A7704
:1099F000280070BD01290CD10223102243700021E0
:109A00000C3001F02DFC305910213530FFF74BF9A7
:109A1000EEE70529ECD10223D118437010220C3057
:109A200001F006FC04233259117F0B431377EAE758
:109A300008251828DCD1053DDAE7C046E465FF1F9C
:109A4000F0B58BB0059143887E4F9E00F459150008
:109A50000493002C15D1012902D000200BB0F0BDD9
:109A6000101D57781678FFF757F9EB68320002930C
:109A70002B7A0499019300903B002000FCF70CFF27
:109A8000EBE7E388049A934201D00820E6E72378C5
:109A9000012B00D1D4E0059B581E092800D9CFE046
:109AA00001F01EFD05CE0A29CC506C859AB2290022
:109AB0000498FFF773FFD1E72000290010224530FA
:109AC00001F0B6FBB9594B78042B02D1013B4B7026
:109AD000C3E70B000A00253335320C310498FFF739
:109AE00095F90498FFF702FA0522431E9841BB59E5
:109AF000C0005A70B2E7200029001022553001F052
:109B000097FB049B4F4C9D00295904980A0006AB13
:109B100055320C31FFF77AF929591022453106A840
:109B200001F0E6FC012808D10498FFF7F7F9059049
:109B3000002804D106222B595A7005988EE7082375
:109B40000593FAE763780C2B7AD1E36E002B03D1EF
:109B50001C2001F0A5FDE066BB59D86E00286FD02F
:109B60001022290001F064FBBB590498DC6EFFF75A
:109B700005FC0D22A076BB595A706EE7E06E0028F6
:109B80005ED063780D2B5BD12B8808220382A91C41
:109B9000123001F04DFBBB599A68517D02221142EF
:109BA00026D0186A407B104222D00C32E4E763785A
:109BB0000E2B45D1236F002B03D1162001F070FD31
:109BC0002067BB59186F002803D01022290001F02C
:109BD0002FFB0F22BB59CFE763780F2B30D1206FBB
:109BE0000622691C103001F023FBBB599A68517D95
:109BF0000422114203D0196A497B1142D5D10021B8
:109C00000498FFF78BFA28E7636F002B0DD0BB5940
:109C1000586F0028F3D01022290001F009FB01221F
:109C2000BB5952425B6F1A61E9E7142001F038FD1D
:109C3000BB5960675B6F002BE9D126E72978DFE726
:109C400007200BE7E465FF1F10B5064C207001F0FC
:109C500047FD06212078FDF791FF0348FEF778FCC9
:109C600010BDC046F765FF1FE98D001100200BB243
:109C700070B50D00834216DA264B187801F000FD0E
:109C8000041E0DD00378922B0ED0A02B37D0224B80
:109C90001878FF283AD0210001F0AAFB002835D11E
:109CA00080200002684070BD43780E2B0BD03E2B05
:109CB000EDD18378052B12D0082BE8D181798088EB
:109CC000FFF7D8FA08E0154B82889A42DFD1836803
:109CD0001878591CFEF7C0FE002817D1D7E7104BA3
:109CE0001B785B0712D50F4B1B68002B0ED09B68AF
:109CF000002B0BD0C289811D80889847ECE7FFF7C5
:109D000041FAA068002801D001F032FC200001F0E7
:109D100017FDC5E7F765FF1F2D43FF1F1820000043
:109D20007164FF1FE065FF1F10B50078FFF712FA9E
:109D300010BD10B50078FFF7FDFA10BD0C234343AA
:109D4000084A10B59B185A68002A03D0012901D18E
:109D5000904710BD9B68002BFBD00029F9D1984794
:109D6000F7E7C0461466FF1F01238340094A10B578
:109D7000946B1C439463506B98435063D46B2000E6
:109D80009843012901D120001843D063116B0B4384
:109D9000136310BD00800040F0B500240127154B6F
:109DA00085B0DA6B144E03921A6C0192DA64019B4F
:109DB000E3403B4217D0039DE5403D400295E5B2AC
:109DC00002992800FFF7BAFF316A736A002908D0A8
:109DD0003900002B01D0029979402800FFF7C4FF19
:109DE00001E0002BF9D101340C36172CDFD105B07E
:109DF000F0BDC04600800040F865FF1F064B012102
:109E00005A68C2400A4204D01B68C3401800084088
:109E100070471B6DF9E7C046008000400122064BE9
:109E20008240002903D0D9680A43DA607047D968B4
:109E30009143D960FAE7C0460038004030B50324AA
:109E400044430F4BE25C1B199C785D7801232D1B6A
:109E50000135AB40013BA340A140DB430C0012287D
:109E600007D808499200521811681940214311601F
:109E700030BD054A11680B4023431360F8E7C04624
:109E8000C7BA001108F0004014F00040C21F70B5BE
:109E9000D4B20623092C0BD80125084C9540002983
:109EA00008D00021FFF7CAFF23682B43236000235B
:109EB000180070BD2368AB43F8E7C0460038004087
:109EC000214BF0B51B185B78022B21D103244443AE
:109ED0001E4A1F4EA35C121994780122150085407A
:109EE000B76B013CE4B23D43A240B563194C122864
:109EF00015D89B0000290CD117495B1899680A43B3
:109F00009A600123205C154A834011680B4313605B
:109F1000F0BD11495B18996891439960F1E70E4BC8
:109F200000290DD159690A435A61225C1328E8D0EF
:109F30000123203A93400A49086803430B60E7E78E
:109F4000596991435961F0E7F865FF1FC7BA0011DD
:109F5000008000400CBB001100F00040A0F0004069
:109F6000A4F00040F8B500241B4E1C4D1C4B1B5D9B
:109F7000012B1FD1194A9269E2401A420BD00122EB
:109F8000B25693402200143AD2B2022A09D8154997
:109F90004A6913434B61013402360C35172CE5D165
:109FA000F8BD0022B2560F499200521891680B4337
:109FB0009360F0E7022BEED1E7B23800FFF71EFF07
:109FC00001235840C1B23800FFF77AFF3800FFF78D
:109FD00015FF6877DFE7C04699BA0011F865FF1FE3
:109FE000F965FF1F00F00040012202388240054B56
:109FF000002903D059690A435A617047596991434E
:10A000005961FAE700380040F8B50E0001210F0051
:10A010008740114A0400D368FD43BB43D360831ECD
:10A020008B4201D8FFF7E0FF00212000FFF72EFF51
:10A030000A4A0B4B5168012E05D139431B19516057
:10A040005E700020F8BD2940516002221C19627028
:10A050009A6915409D61F4E7003800400080004097
:10A06000F865FF1F012210B58240074B002906D07A
:10A0700019680A431A600121FFF7C6FF10BD19686D
:10A0800091431960F7E7C046008000400C2370B58B
:10A09000002543430A4A29009B181D70094B040000
:10A0A0001B185D70FFF7B0FF0123A340064928008D
:10A0B0000A681A430A6005490A689A430A6070BD33
:10A0C0001466FF1FF865FF1F348000403080004099
:10A0D00070B504000E00FF2813D003250540FFF7DC
:10A0E000D5FF084AA3089B009B183F22ED00AA4019
:10A0F000AE40196820009143314319600121FFF7F8
:10A100008DFE70BD18380040F8B50C244443134B45
:10A110000500E4186368002B03D1A3681220002B0C
:10A120001AD0022201270E4B00215B195A70280019
:10A130002770FFF769FF63681E1E08D0A3683E0002
:10A14000002B04D02800FFF759FE4640F6B2280045
:10A150003100FFF709FE0020F8BDC0461466FF1F5E
:10A16000F865FF1FF7B5C420FF222B4B800019585C
:10A17000002491433F3A0A431A508022274F52024B
:10A18000274E1A60274B1D5D002D21D0A31E012BE9
:10A1900003D80121E0B2FFF727FF012D18D11F4B93
:10A1A0009B69E3402B4213D0E3B218000193FFF701
:10A1B00025FE01000198FFF755FFE3B2143B022B87
:10A1C0001DD801217156184A8D405369AB43536124
:10A1D0003B7F002B0DD0E5B22800FFF795FF28004C
:10A1E000FFF70CFE7B7F0100834202D02800FFF7BF
:10A1F000A5FD01340C370236172CC3D1F7BD012160
:10A2000000237156F3568D40074A9B009B189A68AD
:10A21000AA439A60DCE7C04600E100E0F865FF1F52
:10A2200099BA0011F965FF1F00F0004010B5012137
:10A230000400FFF7E9FE0123044A002011194B70C6
:10A24000A34091690B43936110BDC046F865FF1FA1
:10A2500070B50E0015000400FFF718FF0C236343D0
:10A26000094A20009B189D605E60FFF74DFFF021BA
:10A27000064B074A8900051E5A5002D02000FFF7FE
:10A2800005FF280070BDC0461466FF1F0000FF1FB9
:10A29000999D001170B5134D07202C78002C1FD10B
:10A2A000982221005200280001F062F80123C42006
:10A2B000FF222B700C4B80001C635C630B4B1C60FB
:10A2C0005C600B4B195891433F3A0A431A50802265
:10A2D00052021A600D20074A074900F0F1FF2000E2
:10A2E00070BDC046F865FF1F00800040A0F0004030
:10A2F00000E100E065A10011659F0011030010B5A9
:10A300000620072B09D8054A137001F019F8D72148
:10A310000020034B034A89005A5010BD5C43FF1FC5
:10A320000000FF1FD91AFF1F70B51D0002240C2961
:10A3300010D8094ACA40D2070CD5FBF72FFF041EDC
:10A3400008D1059A04992800FBF744FFFCF7B2FDF9
:10A35000FFF712FB200070BD1210000030B50D7821
:10A3600002232C009C43184201D02B431C000825DB
:10A370002300AB43284201D02B00234320241D009F
:10A38000A543204201D01C4325002A230D7018420A
:10A3900004D011781E3B0B43137030BD0028FCD154
:10A3A0000C2113788B43F7E7F8B51D0006AB1B882B
:10A3B000140007AA0E000B201778002B27D10A786B
:10A3C000022A49D14A68507811780002244A084389
:10A3D0008018042840D801F083F803121D1B2300C5
:10A3E000F06800F0EDFF021CC0B2B84200D93A1C80
:10A3F000D2B22000F1682A8000F01AFF06E00222A3
:10A40000F3681B882A8023701B0A63700020F8BD44
:10A410000622EEE701232B80F3681B782370F5E713
:10A42000F368002B16D008222A801A8822701A8816
:10A43000120A62705A88A2705A88120AE2709A88C8
:10A4400022719A88120A6271DA88A271DB881B0A6B
:10A45000E371DBE72B80D9E701202B80D7E7C046EB
:10A4600000D6FFFFF7B516000A781D0008AB1F885D
:10A470000C000123022A18D14A6850781178000292
:10A480002B4A0843801803280FD801F029F8022529
:10A490004439E06800F094FFC0B20723B84204D307
:10A4A0007B190193152B02DD0D231800FEBDE0681A
:10A4B0002A003100C01900F0BBFE6B4600209B88CB
:10A4C000E268D0541B4B1B68834203D01B68834255
:10A4D00000D098470023E8E70B23002FE5D1022D99
:10A4E000E2D1737832781B021343E2681380114B78
:10A4F0001B68002BEED01B68002BEBD00120E8E797
:10A500000B23002FD1D1062DCED12A003100E068D7
:10A5100000F08EFEDEE70B23002FC6D1012DC3D144
:10A5200032787533012AC0D8E3681A70D2E7C04682
:10A5300000D6FFFF0468FF1F70B50C001500072848
:10A5400037D800F0CDFF041436361B36242E1820E1
:10A5500015290BD8184E16220021300000F080FE7D
:10A5600022002900300000F063FE002070BD18209A
:10A570000229FBD11288114B1A80F6E7182008290E
:10A58000F4D10A000E48290001F022F9EDE7182065
:10A590000129EBD10B4B10780B49DA69FFF7DEFE8E
:10A5A000E3E718200129E1D1064B10780749DA6B5F
:10A5B000F4E70220DAE7C046EC67FF1FDA43FF1F2B
:10A5C000D043FF1F6043FF1F8843FF1FA843FF1FA7
:10A5D000030010B50020DB0704D50721024A034819
:10A5E00000F08CF810BDC04624BB00116043FF1F73
:10A5F000054A03001068002803D082889A4201D1DE
:10A60000806870470068F6E7FC69FF1F0A8803004E
:10A6100008009A4204D08A8804309A4200D0002070
:10A6200070470000F8B5F22200230D4F0D4E7968F7
:10A63000050042433370994200D07B600A4C0021F0
:10A64000200000F00DFE00231A007C60AB4202D116
:10A6500000203370F8BD01332280DBB2F234F5E71D
:10A66000F46AFF1FF26AFF1F006AFF1F73B56B4693
:10A6700001900600684615001980FCF74DFF041E86
:10A6800011D1002D0FD07689002E11D00C2001F0B1
:10A6900007F800280ED0084A046013688680856099
:10A6A000002B02D11060200076BD1A001B68F7E76E
:10A6B0000224F8E71324F6E7FC69FF1F01210022BA
:10A6C0000A4B10B549420A4C198099809A719A70C8
:10A6D000084B2070012019805A60FFF7A3FF2078F3
:10A6E000FCF778FF0448FDF733FF10BD0C68FF1F2F
:10A6F000FC6AFF1FF46AFF1FA9A70011022310B50F
:10A70000002802D0FFF7B2FF0300180010BD0000C0
:10A71000030010B50020DB0704D50421024A0348DA
:10A72000FFF7A4FF10BDC04638BB0011E043FF1F78
:10A73000F0B50E2687B003930CAB1F8802ABF6185A
:10A740000500080031000292FDF768F804000120BE
:10A75000002C0FD03088FFF74BFF03000E20002B9A
:10A7600008D05E68002E05D021002800039B029AC5
:10A770000097B04707B0F0BD0A4B10B5984207D11B
:10A780000122002352420A808B708A808B7110BD97
:10A79000FFF73CFF0028FAD001235B42038000232F
:10A7A0008370F4E7FFFF0000F8B5050001290AD126
:10A7B000134E00243388F227AB4219D028001149E8
:10A7C000FFF7DAFF06E0022904D10139FDF73EFF69
:10A7D0000028EDD0F8BD3B0063437268D018D35A0F
:10A7E000002B09D03A00002100F03AFD0134E4B218
:10A7F000054B1B78A342EED801235B423380DDE793
:10A80000F46AFF1F0C68FF1FF26AFF1F10B5FFF705
:10A81000FDFE03000020834200D0987810BD0000A8
:10A82000F0B589B01C000EAB80CB03901E8810AB36
:10A830001B78049202930B7A0D00DB0616D42B785A
:10A840000593022B24D00498FFF7D2FE002812D0E3
:10A8500003689C46002B0ED0029B22000193290026
:10A860003B00644603980096A04705E00498FFF774
:10A87000BFFE002802D10E2009B0F0BD8368002B76
:10A88000F9D00A222900039898470028D7D0F3E787
:10A890006B6858781A786B4B000210439842D2D8F4
:10A8A000043B984210D2684B984242D015D8674B6F
:10A8B000C0180128C7D80B20002EDDD1EB681A780C
:10A8C00059683A80200028E0614BC018032800D95D
:10A8D00079E000F005FE846A789E5E4B9842B2D122
:10A8E0000B20002EC8D101233B80EB6831001B7880
:10A8F00023706889013080B2FCF790FF3A88031E0C
:10A900000ED0017802328A183A80428962704289F8
:10A91000120AA27059680278E01C00F089FC06E077
:10A9200004323A8031000422601C00F099FC0020BF
:10A93000A2E70B20002E9FD1EB6807A91E880423F5
:10A940003B80330A300026706370FCF767FF051EFA
:10A9500028D004AB9A890E2304A95B183E49C66827
:10A96000FCF7D0FF00280BD12B783C486A6805998A
:10A97000FBF786FB002803D1012304AA5B42D381A5
:10A980003278022A06D17168201D00F051FC3B8804
:10A9900002333B800E2304AA9B181B88A3701B0A5A
:10A9A000E370C4E704ABDE81F4E70B20002E00D097
:10A9B00062E7E9680398FFF729FF02233B802070D4
:10A9C000000A6070B3E70B20002E00D054E702228B
:10A9D000EB681B883A8023701B0A6370A7E7E8685E
:10A9E00000F0EEFCC2B203000720B24200D243E7FF
:10A9F0000DD00299DBB27118994202DB921BD3B2DF
:10AA00000293029BE9681A003B8089195AE70023E8
:10AA1000F6E70B20002E00D02EE70722EB683A80E5
:10AA20001A7822705A7862705A88A2705A88120A6C
:10AA3000E2701A792271DA886271DB881B0AA371CD
:10AA400075E7C046042900000228000000D8FFFF77
:10AA5000FFD6FFFF03280000FFFF000068BA0011C7
:10AA6000F0B58DB06B460020089120229B5E83429A
:10AA70003DDAA64B187800F003FE071E32D00378AB
:10AA8000B02B2CD10079023816281FD800F090FD89
:10AA900017001E001E001E0031001E0096001E0042
:10AAA0001D011E0052011E0073011E00CD011E007B
:10AAB00050021E001E001E008E021E00E302944B78
:10AAC00094491B8878880B80FBF71AF83800FCF74C
:10AAD0009BFF914B1B68002B01D038009847380032
:10AAE00000F02EFE8020089B0002434018000DB0AD
:10AAF000F0BDEE220021874800F0B2FB0BAA3B7BA1
:10AB00007989388900923A000D32FCF79FFD0400E4
:10AB1000804B1B78002C3FD146E0804B7888059312
:10AB20007F4B4100CB5A0BAE073BDBB2328802931E
:10AB3000002301937B4B210006930093059BFFF7B5
:10AB40006FFE744D002810D1069B3A8A1B889A42EA
:10AB50000BD138000599123000F0CAFC002804D04F
:10AB60002B7862899B00EB185A80162306A81B18C5
:10AB7000328820007989FCF7C5FE2B7804009A0002
:10AB8000AA1851880029C3D00133DBB22B700028EA
:10AB900007D006A9C98A9180634A12889A42BCD814
:10ABA00002E0012149429180002B04D05949788864
:10ABB000FAF7DAFF8AE73E890A2479E000253E8920
:10ABC000574B06937B88069A5B009B5A033B9D423A
:10ABD00002DB002DF0D05BE0162206A812183B7BAA
:10ABE000798900923A0030000D32FCF72FFD059074
:10ABF000002858D04689017A7888FCF7F1FC041EB9
:10AC000044D1464B78880793069B4100C95A454B6F
:10AC10000439C9B206AAD28A06930291019400931C
:10AC20000599079BFFF7FCFD041E2FD1069B3949B0
:10AC30001A88931C002D26D14B807988384B490007
:10AC4000CB5A5119033B8B4220DD059B31485B8970
:10AC500041190B71A91C0135C9B2EDB20591451915
:10AC60001B0A2B71059B2D490433181800F0E0FADC
:10AC70002C4B059A1B88D318DDB22C4B9E4205D075
:10AC80000136B6B29CE749889942D6D0002D0CD047
:10AC9000204C2800618800F003FC20702100788897
:10ACA000FAF772FF12E7059CF0E7002C00D183E76A
:10ACB0007B78142B00D109E716493B794E800B7045
:10ACC0000C717888FAF712FF00E7162406ABE41837
:10ACD00021003889FCF7A2FD011E00D1B7E1788878
:10ACE00022880F4C45002C5B0A4D013CE4B20294D3
:10ACF00000240F4B01940095FFF792FD041E00D035
:10AD000014E129007888FAF74FFFDFE6FC6AFF1F9D
:10AD1000CC42FF1F1468FF1F0868FF1F0869FF1F50
:10AD20004464FF1FF869FF1FCA42FF1FFFFF0000B6
:10AD30001668FF1F162406ABE41821003889FCF7BB
:10AD40006DFD011E00D182E178882288AE4C45005D
:10AD50002C5BAE4D013CE4B202947C89AC4B019477
:10AD60000095FFF75DFD041E00D0DFE02900788824
:10AD7000FAF724FFAAE60025A44B1D803B00F6331A
:10AD80001B78A24A78880792AB4208D99E4B12885A
:10AD90000693069943005B5A013B9A4203DB0799ED
:10ADA000FAF716FF92E616246B00FB18059306AB24
:10ADB000E418059B21001889FCF730FD011E03D122
:10ADC000059B01241E8973E77888924B2288069C94
:10ADD000099343001B5B904E013BDBB202930023BF
:10ADE00000960193099BFFF71BFD041E02D0059BF3
:10ADF0001E895DE77B88069A5B009B5A079A10883C
:10AE000032881218934202DC1B1A013B33807F4CBC
:10AE1000023032880999001900F00AFA2388328832
:10AE200001359B182380EDB2A8E70BAA3B7B7989FB
:10AE3000388900923A000D32FCF708FC0025059095
:10AE4000059B002B04D10A24002D00D16EE060E0A8
:10AE5000059B7888197AFCF7C3FB0100041E63D1B7
:10AE6000694C6C4B788806940993069B4400E45A1D
:10AE7000694B063CE4B20BAE328807930294019111
:10AE800000930599099BFFF7CBFC041E4CD1079B4F
:10AE90005E491B881A1D002D30D14A80059B5B4CF2
:10AEA0005A8963191A716B1C9BB2E318120A1A7142
:10AEB000162306A832881B1879890598FCF722FD0D
:10AEC000FF21AA1C2E1D03350B00059092B2B6B2CD
:10AED000ADB2002803D006ABDB8AD9B21B0AA21898
:10AEE000651911712B714C4D301D2A884949201864
:10AEF00000F09EF92B88F618B5B2A1E74988914277
:10AF000007D17A8806995200525AEB18053A9A42AC
:10AF1000C4DC3E4C2800618800F05AFB2070210000
:10AF20007888FAF75FFED1E5002DF2D13E89BFE6C1
:10AF3000162606ABF61831003889FCF76FFC3D0089
:10AF40000400FA3500282DD0037A9B060CD4002289
:10AF50007B893989788800923A000C32FFF7E8FB48
:10AF6000041E10D03E8915E03088FFF741FB002811
:10AF70001AD08368002B17D02100122278889847B6
:10AF8000041EE4D0EEE72B78002B02D17888FAF784
:10AF900039FE00262B78002B00D097E5002C00D13D
:10AFA00094E585E60124DDE70E24DBE7162506ABF4
:10AFB000ED1829003889FCF731FC041E47D0037ACC
:10AFC0009B0611D4154A7B881188994203D01448F6
:10AFD000814207D11380134BF2261D780023D9B28A
:10AFE000A94221D30924A1E72888FFF701FB002803
:10AFF0002FD08368002B2CD021001222788898470C
:10B00000041EDFD092E7C0464464FF1F1468FF1F90
:10B010001668FF1F0869FF1FF869FF1FF46AFF1F0A
:10B02000FFFF0000F26AFF1F3100594354680133EB
:10B030006018615A0029D2D13C0008342100F22264
:10B0400000F0F6F821007888FAF7E4FD3EE50124E7
:10B050006CE70E246AE71D4B1A887B889A4231D030
:10B060007888FAF7E1FD31E5F2230598516843430A
:10B07000CD18C95A00291FD03B7A012B0BD16C88FF
:10B08000AB887888AA1D0094FFF752FB041E02D0FB
:10B0900000233B722E88F2220021280000F0E0F805
:10B0A00000232B80059B0133DBB20593084B0599E8
:10B0B0001B78064A8B42D7D801235B421380002CB1
:10B0C000CED0F5E5002634000596EFE7F46AFF1FC1
:10B0D000F26AFF1F70B504000E001500FFF796FA24
:10B0E000031E08D131000548FFF790FA0300112034
:10B0F000002B02D01C8000209D7070BDFFFF00005F
:10B10000F8B50B4F06003B780D001400FF2B0ED056
:10B110000A2000F0FDFA011E09D0B12303800023AC
:10B1200046800371C5800481387800F061F9F8BD6C
:10B130002144FF1FF7B50F0008A90600088809A9D8
:10B140000B240988002821D10234022B1ED1557806
:10B1500013782D021D432B008B4301937334002B76
:10B1600014D1FB68300019000093FFF74FFB019CDE
:10B1700085420BD02A0030000099FFF7ABFF041E78
:10B1800004D12A0030007989FFF7BAFF2000FEBD04
:10B19000F0B50E7885B003900AA805880120022E2C
:10B1A0000DD14C682778647824023C43054FBC429B
:10B1B00005D10398DBB201960095FFF7BBFF05B000
:10B1C000F0BDC04602290000034B10B51B68002BE0
:10B1D00000D09847FEE7C046006BFF1F07B501A8E7
:10B1E000FFF7F2FF044A05480021121A00F0C0F8E8
:10B1F000F8F700FBFEE7C046046BFF1F2444FF1F67
:10B2000001B40248844601BC604700BFC135FF1F3E
:10B2100001B40248844601BC604700BFADAE0000E7
:10B2200001B40248844601BC604700BF3D180000DD
:10B2300001B40248844601BC604700BFE94C0100EC
:10B2400001B40248844601BC604700BF8B52010034
:10B2500001B40248844601BC604700BF9DA90000BC
:10B2600001B40248844601BC604700BF154D01008F
:10B2700001B40248844601BC604700BF2526000097
:10B2800001B40248844601BC604700BF193AFF1F61
:10B2900001B40248844601BC604700BF65710100EB
:10B2A00001B40248844601BC604700BF056A000043
:10B2B00001B40248844601BC604700BF017F000022
:10B2C00001B40248844601BC604700BF6130FF1FE3
:10B2D00001B40248844601BC604700BFC12FFF1F74
:10B2E00001B40248844601BC604700BF1D4B010009
:10B2F00001B40248844601BC604700BF8538FF1F87
:10B3000001B40248844601BC604700BF4D38FF1FAE
:10B3100001B40248844601BC604700BF45500000AC
:10B3200001B40248844601BC604700BF1930FF1FCA
:10B3300001B40248844601BC604700BF8D12000082
:10B3400001B40248844601BC604700BFD91AFF1F00
:10B3500001B40248844601BC604700BF4D1F000095
:10B3600001B40248844601BC604700BF0132FF1FA0
:10B3700001B40248844601BC604700BFB70E00001C
:10B3800001B40248844601BC604700BFB14E0000D2
:10B3900001B40248844601BC604700BF6DBC000098
:10B3A00001B40248844601BC604700BF691F000029
:10B3B00001B40248844601BC604700BF012400007C
:10B3C00001B40248844601BC604700BFDD52010061
:10B3D00001B40248844601BC604700BF79180000F0
:10B3E00001B40248844601BC604700BFED4A010039
:10B3F00001B40248844601BC604700BF594F0100B8
:10B4000001B40248844601BC604700BF0539FF1FF4
:10B4100001B40248844601BC604700BF5D170000CC
:10B4200001B40248844601BC604700BF7D18FF1F7D
:10B4300001B40248844601BC604700BF4537FF1F86
:10B4400001B40248844601BC604700BFE9280000FF
:10B4500001B40248844601BC604700BFA946010010
:10B4600001B40248844601BC604700BFF94C0100AA
:10B4700001B40248844601BC604700BFE1170000E8
:10B4800001B40248844601BC604700BF5952010024
:10B4900001B40248844601BC604700BF9136FF1FDB
:10B4A00001B40248844601BC604700BF350E00006D
:10B4B00001B40248844601BC604700BF091B00007C
:10B4C00001B40248844601BC604700BF0D52010030
:10B4D00001B40248844601BC604700BF5522000009
:10B4E00001B40248844601BC604700BF2D3BFF1FEA
:10B4F00001B40248844601BC604700BFCD4C010046
:10B5000001B40248844601BC604700BFC538FF1F34
:10B5100001B40248844601BC604700BFE548000012
:10B5200001B40248844601BC604700BF5147010096
:10B5300001B40248844601BC604700BFEDA500008D
:10B5400001B40248844601BC604700BF2951010094
:10B5500001B40248844601BC604700BFC521000019
:10B5600001B40248844601BC604700BF21240000AA
:10B5700001B40248844601BC604700BFD9490100BC
:10B5800001B40248844601BC604700BFF30E0000CE
:10B5900001B40248844601BC604700BF5933FF1F15
:10B5A00001B40248844601BC604700BF5125000039
:10B5B00001B40248844601BC604700BF413BFF1F05
:10B5C00001B40248844601BC604700BFA54F01009A
:10B5D00001B40248844601BC604700BF090E000068
:10B5E00001B40248844601BC604700BF9D35FF1F7F
:10B5F00001B40248844601BC604700BFC9A90000ED
:10B6000001B40248844601BC604700BF9135FF1F6A
:10B6100001B40248844601BC604700BF156B0100BD
:10B6200001B40248844601BC604700BFC52DFF1F1E
:10B6300001B40248844601BC604700BF2932FF1FA5
:10B6400001B40248844601BC604700BF792DFF1F4A
:10B6500001B40248844601BC604700BFD91B00000A
:10B6600001B40248844601BC604700BFB54C0100EC
:10B6700001B40248844601BC604700BF2146010076
:10B6800001B40248844601BC604700BFF54E01008A
:10B6900001B40248844601BC604700BF75A90000A0
:10B6A00001B40248844601BC604700BF3D4B010025
:10B6B00001B40248844601BC604700BF456B0100ED
:10B6C00001B40248844601BC604700BFC56D01005B
:10B6D00001B40248844601BC604700BF291C000039
:10B6E00001B40248844601BC604700BFC92600007F
:10B6F00001B40248844601BC604700BF55490100BF
:10B7000001B40248844601BC604700BF014C0100FF
:10B7100001B40248844601BC604700BF1D4D0100D2
:10B7200001B40248844601BC604700BF851F000089
:10B7300001B40248844601BC604700BFDD660100D9
:10B7400001B40248844601BC604700BF434D01007C
:10B7500001B40248844601BC604700BF055E00009A
:10B7600001B40248844601BC604700BF8552010015
:10B7700001B40248844601BC604700BF7139FF1F15
:10B7800001B40248844601BC604700BF3555000043
:10B7900001B40248844601BC604700BFD92FFF1F97
:10B7A00001B40248844601BC604700BF311B000061
:10B7B00001B40248844601BC604700BF090E000086
:10B7C00001B40248844601BC604700BF45510100F6
:10B7D00001B40248844601BC604700BF810E0000EE
:10B7E00001B40248844601BC604700BF5118FF1FE6
:10B7F00001B40248844601BC604700BFED39FF1F19
:10B8000001B40248844601BC604700BF3938FF1FBD
:10B8100001B40248844601BC604700BFC94A010028
:10B8200001B40248844601BC604700BFB352010026
:10B8300001B40248844601BC604700BF193BFF1FAA
:10B8400001B40248844601BC604700BFC51D00002A
:10B8500001B40248844601BC604700BF11470100A3
:10B8600000010103020303030403050206020702A9
:10B87000080209000A030B030C020D000E030F035C
:10B88000100311031303140315001600CD3B001120
:10B89000013C00110000000002000000A2B80011ED
:10B8A000192A0F180A000000F1590000FD240000B9
:10B8B00041460100597C00116D9C0011C1700011BE
:10B8C0005D7A00116D52001161AA0011E14E001164
:10B8D000C13D0011F13E00110000000016160000ED
:10B8E00002000000ECB80011F4FFF3FFD2FC0000EE
:10B8F0003140001100000000000000005475796123
:10B900000042312E3400303031340067697468757C
:10B91000622E636F6D2F7076767800425448303116
:10B92000000000000200000038B90011292A282A6E
:10B93000272A262A252A242A0A180000E2040000C1
:10B940007102000078EC0000744000001027000035
:10B9500060F0000006640000204E000000000000BF
:10B96000050000001F501D00023CB400000114003F
:10B970001400000081020000303132333435363794
:10B9800038394142434445460000000071560011D9
:10B99000C55600110000000002000000A4B900110B
:10B9A0006F2A6E2A1A18000001A000000000000093
:10B9B0006410B71DC8206E3BAC30D9269041DC76B0
:10B9C000F4516B6B5861B24D3C7105502083B8ED5A
:10B9D00044930FF0E8A3D6D68CB361CBB0C2649B7E
:10B9E000D4D2D38678E20AA01CF2BDBDFB349B5FA3
:10B9F000800000800010000000000000C35C001107
:10BA00004D730011E75C0011557700116B5D00115B
:10BA10002B770011E15D001101770011335E0011F9
:10BA2000C97800119B5E0011C9780011CD5E00112C
:10BA300083780011E15D0011B9760011595E0011A3
:10BA40006178001100000000000000003F5F00115D
:10BA500061780011A15F001165730011052A042AA5
:10BA6000012A002A022903280128002801180018A9
:10BA7000000000000000000000000000000000873F
:10BA80000101020102010102010203030401030199
:10BA9000010101010303020103000D000E0010006B
:10BAA000110013001401070108010A010B011C0118
:10BAB0001D02040205020702080219021A021C02F2
:10BAC0001D0301030203170002010005040008071B
:10BAD000000B0A001716001D1C01020101050401DC
:10BAE0000E0D011110011413011716011A1902028B
:10BAF00001020B0A020E0D02111002141302171696
:10BB0000030504030807030B0A030E0D00010203DB
:10BB100007090A0B0E0F101112141718191A1B1F00
:10BB200020212200A9A3001165A40011000000003B
:10BB3000020000006EBA00110000000091B1001177
:0CBB400000000000020000006CBA0011C0
:020000041FFFDC
:1000000000000000293D0011A8B80011A4B800119B
:100010003061FF1F00000000000000000000000031
:1000200000000000000000000000000000000000D0
:1000300000000000000000000000000000000000C0
:1000400000000000000000000000000000000000B0
:1000500000000000000000000000000000000000A0
:100060000000000000000000000000000000000090
:100070000000000000000000000000000000000080
:100080000000000000000000000000000000000070
:100090000000000000000000000000000000000060
:1000A0000000000000000000000000000000000050
:1000B0000000000000000000000000000000000040
:1000C0000000000000000000000000000000000030
:1000D0000000000000000000000000000000000020
:1000E0000000000000000000000000000000000010
:1000F0000000000000000000000000000000000000
:1001000000000000000000000000000000000000EF
:1001100000000000000000000000000000000000DF
:1001200000000000000000000000000000000000CF
:1001300000000000000000000000000000000000BF
:1001400000000000000000000000000000000000AF
:10015000000000000000000000000000000000009F
:10016000000000000000000000000000000000008F
:10017000000000000000000000000000000000007F
:10018000000000000000000000000000000000006F
:100190004D32FF1FAD30FF1FC1660100000000009F
:1001A000000000000000000000000000000000004F
:1001B000000000000000000000000000000000003F
:1001C000000000000000000000000000000000002F
:1001D000000000000000000000000000000000001F
:1001E000000000000000000000000000000000000F
:1001F00000000000000000000000000000000000FF
:1002000000000000000000000000000000000000EE
:1002100000000000000000000000000000000000DE
:1002200000000000000000000000000000000000CE
:1002300000000000000000000000000000000000BE
:1002400000000000000000000000000000000000AE
:10025000000000000000000000000000000000009E
:10026000000000000000000000000000000000008E
:10027000000000000000000000000000000000007E
:10028000000000000000000000000000000000006E
:10029000000000000000000000000000000000005E
:1002A000000000000000000000000000000000004E
:1002B000000000000000000000000000000000003E
:1002C000000000000000000000000000000000002E
:1002D000000000000000000000000000000000001E
:1002E000000000000000000000000000000000000E
:1002F00000000000000000000000000000000000FE
:1003000000000000000000000000000000000000ED
:1003100000000000000000000000000000000000DD
:1003200000000000000000000000000000000000CD
:1003300000000000000000000000000000000000BD
:1003400000000000000000000000000000000000AD
:10035000000000000000000000000000000000009D
:10036000000000000000000000000000000000008D
:10037000DDB10011000000000000000000000000DE
:10038000000000000000000000000000000000006D
:10039000000000000000000000000000000000005D
:1003A000000000000000000000000000591AFF1FBC
:1003B000000000000000000000000000000000003D
:1003C000000000000000000000000000000000002D
:1003D000000000000000000000000000000000001D
:1003E000000000000000000000000000000000000D
:1003F00000000000000000000000000000000000FD
:08183800106FFF1F4118FF1F94
:10184000024981F3088802F02FFA0000106FFF1F91
:1018500010B502F069FA072804D0122808D002282F
:1018600008D010BD044A0420136B01331363F8E75A
:101870000220F6E71420F4E7EC64FF1FF8B5070038
:101880000C0026002500503630785135002804D150
:101890000300287058342370F8BD2978CA00481E08
:1018A0008141A3183800A25C5B68C9B2FFF7D0FF82
:1018B00000280DD12B78DA00A218013350602B706C
:1018C0003378044A013B3370136A01331362D8E75B
:1018D0000123DFE7EC64FF1F5C234343074910B596
:1018E000C9180B0058331B78012B05D1FFF7C6FF31
:1018F000034A936A0133936210BDC0462065FF1FFF
:10190000EC64FF1F10B502F037F9064A01211300FD
:1019100010CB4942D967044B136002F07DFB2000D5
:1019200010BDC04600E100E01000100010B504003A
:1019300002F022F9024B1C6002F06EFB10BDC046A3
:1019400000E100E0431E5A425341A022F0B5D2010B
:101950005B421340154D164A40019B182A18127E0F
:101960008BB00191002A1BD01A000832D46F0022DC
:10197000E6B206AFE4B294420EDC2818C369002B2D
:1019800008D0019902AA117106AA049202AA16733C
:1019900003A898470BB0F0BD1978B9540132EAE7B3
:1019A0001A7D1A7806AB01261A70E6E7AC67FF1FAE
:1019B00000400040F0B5254B04004001C25C85B0FA
:1019C000002A2BD01A18117E002927D0917E0029D9
:1019D00024D01179022921D11689D788D168F51B25
:1019E000ADB22A1C102D00D9102292B2BE4217D1DE
:1019F0001818012303710023C269C38003819A422E
:101A000006D06846032103730171029301A8904731
:101A10000820002C00D0192001F0FEFA05B0F0BD1E
:101A2000013C65426C41A0256442ED012C40084D0B
:101A30001B186419074D0633013A92B2AA42EDD041
:101A40001888461C1E80085C2070F5E7AC67FF1FF5
:101A500000400040FFFF00000F220E4B10B59868B9
:101A6000104002380A280BD802F060F80D0A0B0A61
:101A70000A110A0A0A0A060002210020FFF762FF83
:101A800010BD0121F9E70020FFF794FFF8E7DB6FB5
:101A9000F6E7C046004000400F220E4B10B5986894
:101AA000104002380A280BD802F040F80E0A0B0A40
:101AB0000A120A0A0A0A060002210120FFF742FF61
:101AC00010BD01210800F9E70120FFF773FFF7E7D8
:101AD000DB6FF5E70090004013B5334C2378072BFC
:101AE0003DD8324B1A78324B002A39D180221968FE
:101AF00052020A431A60252001F0C4FE20232D4A19
:101B000011680B43802113606B460422C9050868E5
:101B10000733104228D080210422C905C86810422A
:101B20002ED080212020C905CA688243CA601422B1
:101B30001A701A78002A2FD18021C905C86820326E
:101B40000243CA6014221A701A78002A28D11A4B4C
:101B50001A7D22785A601D221A705932DA6013BD3C
:101B60001A6816490A40C5E7086802430A60142249
:101B70001A701A78002ACED01A78013AD2B2F7E752
:101B8000C8680243CA6014221A7019784A1ED2B279
:101B90001A700029F9D1C4E71A78013AD2B2C7E71E
:101BA0001A78013AD2B2CEE75C43FF1F2444FF1FEC
:101BB0003CF000405443FF1F00200040FFFFFEFFA9
:101BC000564B70B51B68012B03D1554A936D0133F9
:101BD000936502F039F9534B534A1860534B544CF8
:101BE0001A600123534A1360534A13602378002B71
:101BF00006D006225149524802F046F800232370CD
:101C0000504A514B10681B78C1B2002B0ED14F4C7B
:101C1000C0B223785BB2002B4FDB237824785BB211
:101C200064B21B0424021B191B1813600B1C5029DF
:101C30004ED95023464A47491078DBB2FF2202288A
:101C40004BD10868444C454D267890432A789642FB
:101C500054D9227824782E78023B5D10A31B6B4365
:101C60005201D31A10335B111843086002F0CCF90B
:101C7000031F012B45D83A4B1B78002B06D0394B5C
:101C80001B78002B02D0002002F06EF9A122364B07
:101C900092009978354B4A431B689B188322920027
:101CA0009B181B78033B012B03D8AF20400001F0A9
:101CB00093FF01222E4BDA8270BD237824785BB229
:101CC00064B2FF33FF341B0424021B190138ABE755
:101CD000CAB2022AAED20223ACE70868254C264DD0
:101CE000267890432A78964208D9227824782D784D
:101CF000023B5B10641B63435201B2E72378DBB203
:101D0000B2E70228D5D11D4B1B78013B022B03D92A
:101D10001B4B1B78022BCCD16C20C8E79809FF1F06
:101D2000FC0FFF1F2464FF1FFF3F0000141003403F
:101D30002864FF1F0C10034000100340D50BFF1F49
:101D40007211FF1FB40003408C09FF1F680AFF1FB8
:101D5000490AFF1F94000340460AFF1F470AFF1F5E
:101D6000F908FF1F2209FF1F300DFF1F3409FF1F55
:101D7000BC0BFF1F440AFF1F450AFF1F1C09FF1F62
:101D80002309FF1F10B502F037F80022014B1A801B
:101D900010BDC0462064FF1F10B502F015F8A12148
:101DA000054A89009478054A61431268044B521829
:101DB000528C1A8010BDC046300DFF1F3409FF1F22
:101DC0002064FF1F10B50D4B0D4A9978A1239B008D
:101DD0004B431268D218531DD97F0A4B1B88994276
:101DE00009D2441C07D0C82805D0D2695B1A5A43CF
:101DF000054B5343C01802F08FF810BD300DFF1F84
:101E00003409FF1F2064FF1F7102000070B5244DCC
:101E10002B68002B28D002F00FF82B68D8402B68D5
:101E20000400002B27D002F0B7F82B68D8401D4BD8
:101E30001D4A9978A1239B004B431268D118D25CAC
:101E400091239B00002A20D0CA580132CA50174B58
:101E500017491B680868834214D3D23B181A012A19
:101E60001AD0144B186070BD01F0E6FF124B1968D0
:101E700002F0DAF8D3E702F08FF80F4B196802F09E
:101E8000D3F8D4E70D495B18E8E7CA500C4B1B6840
:101E9000DB68E418201AE4E7F530FF30E1E7C046DC
:101EA0001C08FF1F300DFF1F3409FF1F9C09FF1F77
:101EB0002464FF1FA009FF1F1808FF1F2DFF3F000C
:101EC0002C64FF1F70B504000D00282916D10300F3
:101ED000A433C2881B889B1A0B4A9BB293420DD92C
:101EE00006006A3605223100653002F07DF80028D0
:101EF00004D13100200001F0D7FF70BD290020007F
:101F000002F06AF8F9E7C046FE7F0000F8B5050068
:101F1000012001F0A9FE134CA36AA26A9342FBD1EF
:101F2000114E336001F070FF104903000860104843
:101F3000426894460F4A17680022BC4501D24268A5
:101F4000BA1A0D4802603268AD18A422E562606AD0
:101F5000520302436262094A1278002A01D00F3B01
:101F60000B60F8BD00F00040340AFF1FE408FF1FBB
:101F700028100040180AFF1F1C0AFF1F1C09FF1F22
:101F800070B580241025E405A3682B43A36001F0FD
:101F900023FFA368AB43A36070BD0000F7B5160034
:101FA00080221C001023D2050191916805000B438B
:101FB000936000225A4BD7301A6001F0D5FE9D2362
:101FC0002A002F009B00EB58CA3201210092FC37F7
:101FD000002B01D00021009A386801F0B5FE2900DD
:101FE000009BCB311A784F4BD3351A604B780A7867
:101FF0001B0213438A7812041A43CB781B0613433F
:10200000494A1BBA13604B790A791B0213438A7938
:1020100012041A43CB7931001B061343434A1BBAFF
:1020200013606B782A781B021343AA7812041A43B0
:10203000EB781B0613433E4A1BBA1360019A330226
:1020400013433C4A13603C4B22001B1B9C46032954
:102050003DDCB3089A0013005142B21A032A46D15C
:10206000354AE018511A827840781204000202437F
:10207000E05C043302430A600022FF2B4BDDF022B8
:102080002E4B12011A600F222D4B1A602D4A136835
:10209000002BFCD00023224A27491360091B321D64
:1020A0000B191B68043A180A23706070180C1B0E79
:1020B000A070E3700434002AF2DC802210213B6817
:1020C000D20501333B6093688B439360F7BD634651
:1020D000D578981893782D061B042B43157804396E
:1020E0002B43557804322D022B430360AFE7022ABD
:1020F0000AD1114AE05C511AE218527812020243E6
:102100000A6004339BB2B7E7012AB5D10A4A521AD2
:10211000E15C1160F5E7084959180A600433ACE73F
:10212000000004403C0004403800044034000440F7
:10213000300004400C00044000010440040004404E
:102140001000044014000440F7B5150080221C0064
:102150001023D2050091916807000B439360002380
:10216000654AD730136001F0FFFD9D233E009B00C0
:10217000F9583B00CA363200FC33002900D07FE01A
:10218000586801F0E1FD390032785C4BCB311A60C0
:102190004B780A781B0213438A78AC4612041A4320
:1021A000CB78281D1B061343554A1BBA13604B7985
:1021B0000A791B0213438A7912041A43CB791B064E
:1021C0001343504A1BBA13604B7A0A7A1B0213431B
:1021D0008A7A12041A43CB7A21001B0613434A4A17
:1021E0001BBA1360009A2B021343484A1360220063
:1021F000474B1B1B0093009BCE785B1801938B7899
:1022000036061B0433430E78043833434E780431CA
:1022100036023343019E33600328ECDC0321A80817
:10222000431C9B002940800003292BD13849E51825
:102230005E18A9786D78E35C09042D0229431943DF
:102240003160030008330021FF2B2DDD314B324973
:1022500019600F21314B1960012327490B60304B66
:1022600019680029FCD006211B680B40042B20D0E4
:1022700080220020D20593680A318B439360FEBD13
:1022800001217DE7022908D121495D18E11849782B
:10229000E35C090219432960D3E70129D3D11C4922
:1022A0005918E35C0B60CCE7194818180160043337
:1022B000CAE7002310490B606346002B0CDC3B008F
:1022C000FC335A68102101325A608022D20593688B
:1022D00001208B439360D2E7009B9B181B68190A6F
:1022E00013705170190C1B0ED37004235B42917054
:1022F0009C440432E0E7C046000004403C00044037
:102300003800044034000440300004400C00044015
:102310000001044004000440080F000010000440C5
:102320001400044070B5061E19D002225A4B9B7946
:102330009343012B13D1594B1A78FF2A0FD15A78A6
:10234000FF2A0CD19A78FF2A09D1DA78FF2A06D120
:102350001A79FF2A03D15B79FF2B00D199E0504B0A
:102360000C201A78012A08D000224E4D1A702978C4
:102370000B00093B042B01D8212070BD4B1F012B02
:10238000FAD9454CA37B042B00D982E0A279032A19
:1023900000D97EE09A1ED2B2012A02D860881F2896
:1023A00077D9002E56D0012E73D1A0880128E3D012
:1023B000002907D1581E032803D801F0B7FB1217D4
:1023C00015122E702978481E032811D80025364B87
:1023D0001D602823237501F057FDA84227D0A58052
:1023E000CAE702212970EDE70421FBE70321F9E7A1
:1023F00007390129C0D82D490968C96A8906BBD5A2
:102400002B4908780028B7D1012A01D9002BB3D174
:1024100002230B708021274D2633890128782375EC
:1024200001F00AFE80212878890101F0B5FB012323
:10243000A380214B1B78002B0AD0FA2280211F4B4E
:1024400092001B8809025A431A4B187801F04CFC81
:10245000002092E701F090FB2B78A680073B012B30
:1024600003D917482E7001F05FFD114B114C1A78FB
:10247000002A06D080210022207889011A7001F0FC
:10248000DBFD01F0C9FD80212078090201F0D4FDB7
:10249000DEE7122071E7C046A60BFF1F6B09FF1F86
:1024A0001A09FF1F1C09FF1F4809FF1F2C64FF1F8B
:1024B0002309FF1F1B09FF1F2109FF1F2C09FF1FF5
:1024C0000010004010B5002901D001F0E5FB10BD5F
:1024D000F7B5604B01919978A1239B004B435E4A6D
:1024E000060014681022E418D6235B00E058362357
:1024F000FF33E35C00279343222B41D1574B0F3A24
:102500001A600760012501F02FFB019B1880E8236A
:102510005B00E35C002B01D0B34258DD0023504F39
:10252000FB70AD33FF33E3581A68002A03D09B8851
:10253000DB439B071DD03823FF33E35C002B18D00F
:102540009B235B00E35C002B13D1D133FF33E35CAF
:10255000B3420EDAA4235B00E15AE018090A023103
:1025600001F02AFD23000122FE33013E01351A87C6
:10257000FA70E8235B00E35C002B2AD0A8B2FEBD12
:1025800003683D00002BBED081880430090A023167
:1025900001F012FDD6235B00E3581F60B2E7230071
:1025A000B133BA00FF339858013781880430090AE3
:1025B000023101F001FDE8235B00E35CBB42EEDC8D
:1025C000E822F61AED1800235200A354A6E70027CC
:1025D000F1E7200001F020FB00281FD0002E1DDDB8
:1025E0007319882647190193B600200001F06CFB8F
:1025F0005A30800020184068013581880430090A6B
:10260000023101F0D9FC200001F0F6FAA3590133A0
:10261000A351BD4202D0019B9D42E6D1114BE35C28
:10262000002BABD095239B00E35C002BA6D00E4B78
:10263000E15A0029A2D00D4AA35C994202D9013384
:10264000A3549BE700231A212000A35401F084FA2D
:1026500094E7C046300DFF1F3409FF1F00140340EC
:10266000E010FF1F5A020000720200005E0200002C
:102670000D4970B54A6E0D4CD2038B69D20BA24244
:1026800006D80B4D0224AA4204D901F02DFC70BDDE
:1026900002246442E21815007E2425402242F4D030
:1026A000A3432B438B61F0E700F000400A200000B9
:1026B000FC1C0000F8B51D4B1D4F1A78002A10D1E4
:1026C000BA7B002A02D101321A7003E0032AFAD041
:1026D000022AF8D001F0D8FB00220120154B1A7015
:1026E000F8BD154B154D1C68154B9E7801232B70BA
:1026F0002878C0B200F0A2FBBB7B002B0BD101F00D
:1027000093FBA1239B007343E41883239B00E418ED
:1027100023782B70E4E7032B02D101F0A5FBF0E74F
:102720000020022BDCD101F0C7FAEAE71C09FF1FE9
:10273000A60BFF1F2309FF1F3409FF1F490AFF1FB4
:10274000300DFF1FF0B587B00EAD2F780FAD2D788F
:102750000593AC46634614000E4D0CAA12782E78F1
:1027600003930D9B009201932200059B029701F0B9
:10277000C3FB2E70012C01D0042C08D18022064905
:102780008B889343054A1278D20113438B8007B09C
:10279000F0BDC0461C09FF1F6C11FF1F7809FF1F09
:1027A0000B001B3B70B504003020E02B0DD813004C
:1027B000E025493BFF3B9BB2ED00AB4205D8034B04
:1027C000200019825A8201F01FFA70BD8410FF1F89
:1027D00010B501F039FB054B00205B68052B04D9CF
:1027E000034A5268D20200D4980810BD001000407D
:1027F000FCE100E070B501F0BFF90D4B1B68FC3344
:10280000DC691D6AFFF7E4FF6419844204D2094BB6
:1028100001241B68002B07D004220024064B1A70E9
:10282000064A93690133936101F0F6FB200070BD05
:102830002C64FF1F9809FF1F2309FF1FFC0FFF1FB8
:1028400070B50C4D2B68FC335C6A01F095F9FFF70D
:10285000BFFF2B680025FC339B6AE318834204D238
:10286000054B1B68AB4200D1051B01F0D5FB2800CE
:1028700070BDC0462C64FF1F9809FF1FD722044B70
:1028800092009B5810B5002B00D0984710BDC04651
:102890000000FF1F10B501F0D3F8FFF7EFFF274945
:1028A000274BCA6D274C1A4084235B001343CB652A
:1028B000254B1B68186A01F0D7F9244B244A1A608B
:1028C000244B254A1A60A022244B52001A60244B44
:1028D000187801F0E1FA2000224901F0BDF9002347
:1028E000A3600233A360204B2049236003232048C8
:1028F000A36001F0B1F910221E4BFF201A60802264
:1029000052031A60802292031A60802212041A6015
:1029100001F02AFB012001F047FBFA20400001F002
:10292000DBFA582001F058F9134801F0EDF90120C5
:1029300001F04AF9072001F08FFB10BD00F00040C4
:1029400000FEFEFF141000402C64FF1F0000034037
:102950000180063DBC00034034080000A400034091
:102960004A0AFF1F71020000C3090000FFFF3F0079
:102970002810004000E100E030750000674E336829
:1029800088331B6883F3088801F02EFA644A65498E
:10299000136800200B401360634B644A1B6893422A
:1029A00000D1A6E001F050FB0221614A13688B437D
:1029B0001360FFF76FFF5F4B5F4C1878C0B201F0F8
:1029C0008BF90023A3600233A3605C4B01202360DA
:1029D00001F04AF90323A36001F0E6F8040001F0D6
:1029E00033FA050001F0E0F8554B186001F08CFA5D
:1029F000544B1968621A531EA14200D21300802260
:102A0000D203934201D39B029B0A3268D16AC90761
:102A100000D471E04C491C0C09689BB24C435943EB
:102A20002402090A641803264849FC3293680A689C
:102A300047489B1A474A0768126847499B18474A04
:102A40009A1833409208DB190A600360042B03D9FB
:102A5000013233400A6003600E684149A619300014
:102A600001F0E2FA3F4F3E493B68C3183B6030003B
:102A7000019301F041F93C4E306808183849306044
:102A8000884205D9019B01333B6001F035F9316083
:102A900001F0C2F9354B1B78002B0DD001F0D4F9B1
:102AA000334B621B196812188A4232D24919091B2A
:102AB000091A304801F0D0F82F4E337A002B0ED08F
:102AC00001F0C2F9621BF1681218914224D9491928
:102AD000091B091A294801F0BFF800233372284B5B
:102AE00083F3088801F050F8002001F0ADFA01F0FE
:102AF000EBF901F0A9FA5CE7DC0199000234641AF1
:102B00005900641A09214B438033CB40A408E418D0
:102B100089E7FA218900CCE71A49DBE72C64FF1F1B
:102B20001CF00040FFFFC1FF0C0AFF1FB64121034C
:102B300010000040490AFF1F14100040C3090000A4
:102B4000100AFF1F340AFF1F380AFF1F200AFF1F49
:102B5000280AFF1F1C0AFF1F240AFF1FC4090000C8
:102B6000710200006008FF1F2C0AFF1F1C09FF1FD5
:102B7000E408FF1F00100040740BFF1F3C100040D2
:102B800000000020DC050000A022054B92009B58AD
:102B900010B5002B01D0984710BD01F04DF8FBE7B0
:102BA0000000FF1FA122054B92009B5810B5002B7F
:102BB00001D0984710BD01F03FF8FBE70000FF1F70
:102BC000A222054B92009B5810B5002B01D09847CC
:102BD00010BD01F031F8FBE70000FF1FA322054BF9
:102BE00092009B5810B5002B01D0984710BD01F002
:102BF00023F8FBE70000FF1FA422054B92009B581F
:102C000010B5002B01D0984710BD01F015F8FBE777
:102C10000000FF1F70B501F017F94F4B186001F06D
:102C200003F80400C30702D401F0C6F870BD002207
:102C30004A4B1A604A4B18780138042829D800F00A
:102C400075FF0320181C2400200001F095F80128CE
:102C5000ECD0444C2378042B6ED101F02DF90028E0
:102C6000E4D001F069F8582000F0B6FF0223237089
:102C7000DCE7200000F0E8FFE9E7200001F06CF855
:102C8000E5E7200001F0E8F8E1E7200000F0F4FFBC
:102C9000DDE701F0B9F90500012808D1324B1B78B6
:102CA000053B012B03D82000FFF76EFFD1E72D4B2A
:102CB0001B78022B01D0052B20D1022D28D12B4BC4
:102CC0009B7BAB431CD12000FFF76CFF264B187891
:102CD0000128BED16405BCD4244925224B7B034284
:102CE00005D1233A13405A42534126331A000B7D33
:102CF0009342AED9322001F02FF9AAE7022D07D175
:102D0000194B1B78052B11D12000FFF759FFDDE788
:102D1000012D0BD1012B03D12000FFF75FFF98E7B6
:102D2000062B03D12000FFF767FF92E7200000F099
:102D300083FF022D8DD1C9E7032B04D10C4B987C66
:102D400001F09AF872E7072B00D06FE7094B987BE8
:102D500001F01AF96AE7C0469C09FF1F9809FF1F96
:102D60009009FF1F2309FF1F1C09FF1FA60BFF1F50
:102D7000BC0BFF1FD40BFF1FFA210A4B0A4A490064
:102D80001A640A4A5A500A4A04395A50094A083100
:102D90009A64094A5A50094A5C315A50084ADA661C
:102DA0007047C0460000FF1F4527FF1F4128FF1F37
:102DB000F527FF1F2523FF1FB526FF1FC51DFF1F7A
:102DC000991DFF1F10B500F099FE10BDF7B50B0C53
:102DD000FF270122009300233C001E001D009446A3
:102DE000019089B262469A40100008401841361896
:102DF000B6B2FF2F02D1012E00D19FB2009802403F
:102E00001A41AD18ADB2FF2C02D1012D00D19CB2F8
:102E10000133102BE6D10320012E07D1012D04D15F
:102E2000019B2401E4191C700138FEBD102EFCD159
:102E30000238102DF9D00230F7E700008023F7B5F3
:102E40009C46264B264F01932649274A274D284C5E
:102E5000284B02281AD1604638600868264E304058
:102E6000802636033043086001990978002909D18A
:102E70001660224A2A60224A2260E02219689143A1
:102E8000A03A1BE08021C9021160F2E766463E606D
:102E90000F68194E3E408027FF023E430E600199A5
:102EA000097800290DD1176001280ED1154A2A6032
:102EB000154A2260E02219689143C03A0A431A6019
:102EC000F7BD802189021160EEE7E0210F4A02433D
:102ED0002A600F4A22601A688A43F0E74B0AFF1FF4
:102EE000E0000340D800034090000340000003408E
:102EF0005000034040000340FFFFE3FF0280063D17
:102F0000804508220180063D8066082200800698E0
:102F100080550822F8B51E4B80261A680020140040
:102F20003440324232D11A681A4F32431A600122B9
:102F30003B68063093433B6000F096FE0122164D3D
:102F40002B681E432E603B680A2613433B60802794
:102F5000BF00124B1B683B4211D1013EF6B2FF2E5F
:102F600009D17E220E4B1C682B68E40B144093435E
:102F700023432B6005E0082000F076FEE9E7002EF1
:102F8000EFD180222B68600893432B60F8BDC046C8
:102F9000C4F000405CF0004018F0004068F00040D1
:102FA00060F0004010B501F00FF801215820034AED
:102FB00000F002FEFFF7AEFF10BDC046600AFF1F23
:102FC00010B578220021034800F0D6FF00F0B4FFCE
:102FD000002010BD3467FF1F70B5040000F0CCFD69
:102FE00000230C200B4A010059438D18515C002925
:102FF0000DD0A14208D1012300246B7000F0F4FD34
:1030000001F00AF8200070BD01330A2BEBD1122425
:10301000F6E7C0463467FF1F70B5040000F0ACFD52
:10302000002319001D000D4A1078002806D0A04288
:103030000CD1557001310C320A29F5D1002B0AD17F
:1030400000F07AFF00F0E8FF002070BD5078461EC7
:10305000B0411B18EEE700F0C7FDF3E73467FF1F30
:10306000F7B504000C20002384460E4D01926746FC
:103070005F43E85D7E19A04212D000280BD10A4BB5
:103080009C4662461B7808331370019B70707C5518
:103090007160B360FEBD01330A2BE8D10320F9E76C
:1030A0000720F7E73467FF1F3067FF1F8020F8B560
:1030B000484BC0051B68C1248360474BFF251A6835
:1030C000012313434361454BA4001A68444B40213C
:1030D0001A60444B1A68444B1A60444B1A59AA436D
:1030E0001A51C52292009E58AE4331438026995012
:1030F0009F583F49F6010F403E439E509E588027FF
:103100003602360A3043985080201A5900020A408D
:1031100002431A5104341A59364E3F043240802675
:103120003A431A511A5936061202120A32431A51F8
:1031300008341A5980260A4002431A51C3229200C9
:103140009F58B446AF4337439F509F58294E0F4076
:1031500007439F509F5837408026360437438026C8
:103160009F509F5836063F023F0A37439F50C02268
:103170001F59AF433A431A511A591202120A164301
:10318000C6221E5192009C58AC4365462C439C506D
:103190009C5800250C4020439850C72080001A58A6
:1031A000154C1140C02212020A431A50134B1B78CF
:1031B000DB08AB4201DC0020F8BD2378002B06D0F1
:1031C000A368002B00D0984701350C34EEE712209D
:1031D000F2E7C0465843FF1F5443FF1FB0F00040C2
:1031E0002C67FF1FB4F000402867FF1F00E100E0DC
:1031F000FF00FFFFFFFF00FF3467FF1F3067FF1F67
:10320000030010B51F2809D8072200201340072407
:1032100004490A78A24313430B7010BD0023062013
:10322000F5E7C0463067FF1F054B06491B780A6863
:1032300005485B0702401B0B134300200B607047DF
:103240003067FF1F1CF00040FFFFC1FF70B50C2569
:10325000FFF7EAFF0A4B1C780A4BE4086543ED18B8
:10326000002C01D1200070BD2B78002B06D06B689C
:10327000002B00D09847013C0C3DF1E71220F2E70B
:103280003067FF1F2867FF1F1FB5002102220B00B8
:1032900001910091052000F077FD02230B490A6897
:1032A0001A42FCD120230393039B5A1E0392002B46
:1032B000FAD1074A1368002BFCDA0B246C44200077
:1032C000012100F029FD207804B010BD90C8004015
:1032D00000C8004013B504000A4B0193019B002B6A
:1032E00001D1112016BDFFF7CFFF23000340044298
:1032F00005D0052000F0B8FC019B013BEDE718006C
:10330000F0E7C046FFFFFF0707B500F035FC80225D
:103310000821D205936A0191002B01D107399162EE
:1033200002210C4A11600199481E01900029FAD12E
:1033300003311160053101910199481E0190002966
:10334000FAD11160002B02D18022D205936200F0E5
:1033500063FE07BD00C00040F0B52D4C89B0237856
:10336000002B4FD1FEF7CEFA02232A4F03903A6882
:103370001A42FCD120230693069B5A1E0692002B6C
:10338000FAD1254E3368002BFCDA0120FFF7A2FFAB
:10339000011E02D0112009B0F0BD030003220190EC
:1033A000009005AD9F2000F0EFFC0321280000F005
:1033B000B3FC02233A681A42FCD120230793079BEF
:1033C0005A1E0792002BFAD13368002BFCDA012039
:1033D000FFF780FF0028DDD10398FEF7A7FAAA784F
:1033E0006B7811041B020B4329780B4363601300B5
:1033F000113B0A49052B07D801239340A3600B60BA
:10340000012323700020C6E780231B03F6E7C04694
:103410004043FF1F90C8004000C800409808FF1FAD
:103420001E4B30B55A6818781D4B85B0D3185942D9
:103430004B4101210093002300F0AEFC194B1A4AC6
:1034400002259A6300221A6510325A658022C4212F
:103450009D65164B1648D202DA6789004258154B13
:1034600080241A4080231B041343435064234120CB
:103470000393E40500F006FA402000F003FA6562C9
:10348000039D6B1E0393002DFAD103236362FFF7A4
:103490003BFFA562FFF760FF05B030BD4C43FF1F47
:1034A00095FFFEF700C80040050001FF04E100E0C1
:1034B00000E100E0FFFF00FFF0B585B00700FEF778
:1034C00021FA022305002D4C22681A42FCD1202348
:1034D0000093009B5A1E0092002BFAD1284E3368AD
:1034E000002BFCDA0120FFF7F5FE002803D01124A1
:1034F000200005B0F0BD234B2360022322681A424E
:10350000FCD120230193019B5A1E0192002BFAD17A
:103510003368002BFCDA0120FFF7DCFE0028E6D13F
:10352000194B1F60022322681A42FCD12023029308
:10353000029B5A1E0292002BFAD13368002BFCDA50
:103540000120FFF7C7FE0028D1D1104B23600223D2
:1035500022681A42FCD120230393039B5A1E039234
:10356000002BFAD13368002BFCDA0120FFF7B2FE02
:10357000041EBCD12800FEF7D9F9B9E790C8004075
:1035800000C8004001000006A8C8004001800001FA
:1035900010B50020FFF790FF10BD000010B5064BDE
:1035A00018705960FFF73CFF00211320034AFFF712
:1035B00057FD002010BDC0464C43FF1F2134FF1FA4
:1035C000F0B5040085B003920291FEF79BF98822C2
:1035D00063035B0B52051A438023DB059D6A80233E
:1035E000274F0092BA68002601901B039A420CD91B
:1035F000F82326001B041E401C4206D08022214BCB
:1036000052025E6219680A431A60002D0BD100F065
:10361000B3FA02221C4B1A608023DB055A62013A7E
:103620009A6200F0F9FC0023039A934220D1002D06
:103630000AD100F0A1FA144B03221D608023DB05A0
:103640005A629D6200F0E8FC8023BA681B039A422C
:1036500008D9002E06D000220A4B0C495A621A687B
:103660000A401A600198FEF761F9002005B0F0BD2C
:10367000009A0299D2181278CA540133D4E7C0468E
:103680004043FF1F00C8004000C00040FFFFFEFF96
:10369000F0B587B0029103920400FEF733F9019070
:1036A00000F06AFA802302250122234EDB053560F3
:1036B0005D629A6200F0B0FC204F3B682B42FCD167
:1036C00020230493049B5A1E0492002BFAD11C4D14
:1036D0002B68002BFCDA0120FFF7FCFD002802D04C
:1036E000112007B0F0BD2000039A029900F084FC7D
:1036F000022304003A681A42FCD120230593059B5B
:103700005A1E0592002BFAD12B68002BFCDA0120FF
:10371000FFF7E0FD051EE3D100F02EFA802303221F
:10372000DB0535605A629D6200F076FC0198FEF779
:10373000FDF8E0B2D5E7C04600C0004090C80040A8
:1037400000C80040F0B5802489B00600FEF7DAF822
:10375000E405A36A02250393029000F00DFA012309
:10376000304F3D606562A36200F056FC2E4C23682A
:103770002B42FCD120230593059B5A1E0592002B5A
:10378000FAD12A4D2B68002BFCDA0120FFF7A2FDAD
:10379000002803D01124200009B0F0BD244B236081
:1037A000022322681A42FCD120230693069B5A1E4C
:1037B0000692002BFAD12B68002BFCDA0120FFF7D0
:1037C00089FD021EE6D11B4B03211E600300019000
:1037D0000090202000F0D8FA022322681A42FCD17F
:1037E00020230793079B5A1E0792002BFAD12B68C0
:1037F000002BFCDA0320FFF76DFD041ECAD100F098
:10380000BBF980230322DB053C605A629C6200F016
:1038100003FC039B002B01D1FFF776FD0298FEF716
:1038200085F8B8E700C0004090C8004000C80040DC
:103830000100000694C8004007B50002019104226F
:10384000000A01A9FFF724FF0EBD000073B50500B3
:1038500005240B4AA3005B429B1819686B46DE1DCA
:103860003000FFF7B3FA022804D133782B55013C1E
:10387000EFD276BD052CFCD00128FAD10230F8E752
:10388000140900111F2807D8012380228340D20584
:1038900091680B43936070473F2808D8012380222A
:1038A00020388340D20551690B435361F3E75F2809
:1038B000F1D80123802240388340D205116A0B439E
:1038C0001362E8E71F2807D8012280218240C9053A
:1038D0008B6893438B6070473F2808D80122802172
:1038E00020388240C9054B6993434B61F3E75F2859
:1038F000F1D80122802140388240C9050B6A9343E8
:103900000B62E8E71F2810D880230200DB05153A78
:103910001968012A06D820229143196019680A43C0
:103920001A60704701228240F6E73F2811D88023B1
:103930000200DB05353AD968032A06D810229143E4
:10394000D960D9680A43DA60EBE701222038824067
:10395000F5E75F28E5D842238022181A413B8340CF
:10396000D205516A99435162516A0B435362D8E7B9
:1039700010B50400012813D1A022184992050B6844
:103980005B015B0913430B60154B164A1968114024
:10399000154A0A431A60402219680A431A6010BD8A
:1039A0000028FCD101000A2000F0FEF921000B20C4
:1039B00000F0FAF9C0220A4B920019680A4340212C
:1039C0001A601A688A431A60B022044912060B680A
:1039D0005B015B0913430B60E1E7C04614F0004054
:1039E0001CF000407F00FEFF80FD010072B6074A18
:1039F0001368013313600422054B1A600023054A43
:103A000013608022D2055360FEE7C0467808FF1F8E
:103A1000C0F00040C4F0004005490B68002B05D100
:103A2000044A0A6004490A60044A13607047C046A9
:103A3000140AFF1F841E0000380AFF1FC4F0004054
:103A40000023034A1360034A1360034A136070475C
:103A500054F0004040F1004044F10040002310B514
:103A6000184C8AB0009301932378012B27D0694624
:103A7000012000F069FA002817D1009B1249029337
:103A8000019B06AA0393114B02A81B680493104BD9
:103A90001B68059300F0A0F910220E4906A800F05B
:103AA000A3FA002804D1FF23237000200AB010BD20
:103AB0000123094A074902A8237000F08DF901206B
:103AC000F4E7C0463064FF1F1029001108290011D7
:103AD0000C290011202900113464FF1F13B50124A3
:103AE0006946012000F030FA034B00940193FFF780
:103AF000B5FF200016BDC046BB0B000010B5FFF798
:103B00009FFFFFF7EBFF002802D0024B984710BD44
:103B1000FEE7C046E1A2000002B471464908490030
:103B2000095649008E4402BC7047C04602B4714633
:103B300049084900095C49008E4402BC7047C046F0
:103B400003B47146490840004900095A49008E44AF
:103B500003BC70470000000001B40248844601BC69
:103B6000604700BF53B9000001B40248844601BC5D
:103B7000604700BFCD0C010001B40248844601BC7F
:103B8000604700BF75A9000001B40248844601BC2B
:103B9000604700BF7997000001B40248844601BC29
:103BA000604700BF0D52010001B40248844601BCC9
:103BB000604700BF156B010001B40248844601BC98
:103BC000604700BF0167010001B40248844601BCA0
:103BD000604700BFE512010001B40248844601BC01
:103BE000604700BF7912010001B40248844601BC5D
:103BF000604700BF21A9000001B40248844601BC0F
:103C0000604700BF5976010001B40248844601BCF8
:103C1000604700BF116E000001B40248844601BC39
:103C2000604700BF71B0000001B40248844601BC87
:103C3000604700BFBD0B010001B40248844601BCCF
:103C4000604700BFE917010001B40248844601BC87
:103C5000604700BF0934010001B40248844601BC3A
:103C6000604700BF2D6C010001B40248844601BCCE
:103C7000604700BF0189000001B40248844601BCCE
:103C8000604700BFF935010001B40248844601BC19
:103C9000604700BFE94C010001B40248844601BC02
:103CA000604700BFE9D4000001B40248844601BC6B
:103CB000604700BFE5B1001101B40248844601BC71
:103CC000604700BF19FA000001B40248844601BCF5
:103CD000604700BFD9B0000001B40248844601BC6F
:103CE000604700BF8914010001B40248844601BC4A
:103CF000604700BF8B52010001B40248844601BCFA
:103D0000604700BF090E000001B40248844601BCB0
:103D1000604700BF8D11010001B40248844601BC18
:103D2000604700BF3D71010001B40248844601BCF8
:103D3000604700BFE927000001B40248844601BC87
:103D4000604700BF6DF6000001B40248844601BC24
:103D5000604700BF2144000001B40248844601BC12
:103D6000604700BF0534010001B40248844601BC2D
:103D7000604700BF8944000001B40248844601BC8A
:103D8000604700BF0134010001B40248844601BC11
:103D9000604700BF496D010001B40248844601BC80
:103DA000604700BFC56D010001B40248844601BCF4
:103DB000604700BF3D9E001101B40248844601BC2B
:103DC000604700BFDD0A010001B40248844601BC1F
:103DD000604700BFF9ED000001B40248844601BC11
:103DE000604700BFDD3F000001B40248844601BCCB
:103DF000604700BFC9A9000001B40248844601BC65
:103E0000604700BF8D82000001B40248844601BCB7
:103E1000604700BFBD5C010001B40248844601BC9C
:103E2000604700BFD544010001B40248844601BC8C
:103E3000604700BFE9F6000001B40248844601BCB7
:103E4000604700BFE90B010001B40248844601BC91
:103E5000604700BFC95C010001B40248844601BC50
:103E6000604700BFF535010001B40248844601BC3B
:103E7000604700BF75F8000001B40248844601BCE9
:103E8000604700BF4DF9000001B40248844601BC00
:103E9000604700BFA9D8000001B40248844601BCB5
:103EA000604700BFEDA5000001B40248844601BC94
:103EB000604700BF85C1000001B40248844601BCD0
:103EC000604700BF01D7000001B40248844601BC2E
:103ED000604700BF8552010001B40248844601BC1E
:103EE000604700BF8512010001B40248844601BC4E
:103EF000604700BFD1AE000001B40248844601BC57
:103F0000604700BF9D6A000001B40248844601BCBE
:103F1000604700BFC166010001B40248844601BC8D
:103F2000604700BF8937010001B40248844601BCE4
:103F3000604700BFC1A5000001B40248844601BC2F
:103F4000604700BFADAE000001B40248844601BC2A
:103F5000604700BFE1AC000001B40248844601BCE8
:103F6000604700BF6137010001B40248844601BCCC
:103F7000604700BFED6B010001B40248844601BCFC
:103F8000604700BFB70E000001B40248844601BC80
:103F9000604700BFC1F7000001B40248844601BC7D
:103FA000604700BF6D0B010001B40248844601BCAC
:103FB000604700BF6911010001B40248844601BC9A
:103FC000604700BFC115010001B40248844601BC2E
:103FD000604700BFED68010001B40248844601BC9F
:103FE000604700BF51B8000001B40248844601BCDC
:103FF000604700BFCD4C010001B40248844601BCBB
:10400000604700BF9573010001B40248844601BCBB
:10401000604700BFDD0C010001B40248844601BCCA
:10402000604700BF9DA9000001B40248844601BC5E
:10403000604700BF090E000001B40248844601BC7D
:10404000604700BFB352010001B40248844601BC7E
:10405000604700BF016C010001B40248844601BC06
:08406000604700BFF90D0100EB
:10406800020000006ABA00110100000098B80011AF
:104078000200000066BA001101000000A840FF1FFE
:1040880002000000A0B8001101000000B061FF1F8D
:104098000200000064BA0011030000002461FF1F41
:1040A80012000000020000006ABA001101000000BE
:1040B800E0B800110200000066BA0011010000001B
:1040C800DDB8001102000000EAB80011030000008A
:1040D8005F61FF1F0200000064BA001103000000C6
:1040E8007461FF1F0200000066BA001101000000A1
:1040F800DCB8001102000000E8B80011030000005D
:104108003561FF1F0200000064BA001103000000BF
:104118005661FF1F020000006ABA0011010000008A
:1041280024B900110200000066BA00110100000065
:10413800F141FF1F0200000036B900110100000024
:104148001BB900110200000066BA0011010000004E
:10415800F041FF1F0200000034B900110100000007
:104168007C61FF1F0200000066BA00110100000018
:10417800EF41FF1F0200000032B9001101000000EA
:104188000BB900110200000066BA0011010000001E
:10419800EE41FF1F0200000030B9001101000000CD
:1041A80006B900110200000066BA00110100000003
:1041B800ED41FF1F020000002EB9001101000000B0
:1041C80001B900110200000066BA001101000000E8
:1041D800EC41FF1F020000002CB900110100000093
:1041E800FCB80011020202020202000000000000F6
:1041F80016150000054B0011C94A001178B90011C5
:1042080090011D0018001800FFFF070102030405B4
:104218000602010600000000000000000000000087
:104228000000000000000000000000000000000086
:1042380003000000020000006ABA0011010000003B
:1042480098B900110200000066BA001101000000D0
:10425800AC42FF1F02000000A2B9001101000000DB
:10426800AA61FF1F0200000064BA001103000000E9
:104278001464FF1F0200000066BA0011010000006C
:10428800AC42FF1F02000000A0B9001101000000AD
:10429800AC61FF1F0200000064BA001103000000B7
:1042A8000C64FF1F12000000000100000000011153
:1042B800FFFF0000504859360000000000000000D1
:1042C8000B000500F0000000B400002800280028BA
:1042D8003075A000A000A000A00000080008E001C0
:1042E800F000100010001000100010001000500026
:1042F8005000500010001000D0070000000000001F
:104308000F0001000500307507001000010081FF53
:1043180000000000FF000000257000112D6E001144
:10432800BD6B0011FFFF0100FF000000419A001162
:10433800BD970011D5960011000000000000000094
:1043480000000800040000003B0001085902E001D9
:1043580088212800FF000000020000006ABA00114E
:104368000100000030BB00110200000066BA001115
:1043780001000000DD43FF1F0200000062BA0011C7
:1043880001000000EC67FF1F0200000066BA001180
:1043980001000000DC43FF1F0200000060BA0011AA
:1043A80001000000DA43FF1F0200000066BA001196
:1043B80001000000D843FF1F020000005EBA001190
:1043C80001000000D043FF1F180018001D009001D5
:1043D8000200000302020000020000006ABA001195
:1043E8000100000044BB00110200000066BA001181
:1043F800010000002044FF1F020000005CBA001109
:1044080000000000000000000200000064BA001173
:0A441800030000000C68FF1F20FFE6
:040000051FFF184180
:00000001FF
